:020000040800F2
:10000000C08C0020BD010008C5010008C701000820
:10001000C9010008CB010008CD0100080000000064
:10002000000000000000000000000000CF010008F8
:10003000D101000800000000D3010008D50100082C
:10004000D7010008D7010008D7010008D701000830
:10005000D7010008D7010008D7010008D701000820
:10006000D7010008D7010008D7010008D701000810
:10007000D7010008D7010008D93E0008D7010008C1
:10008000D7010008D7010008D701000800000000D0
:10009000000000000000000000000000D701000880
:1000A000D7010008D7010008D7010008D7010008D0
:1000B00063270008F12E0008D7010008D7010008C7
:1000C000D7010008D7010008D7010008D7010008B0
:1000D000D7010008EB3F0008D70100086145000880
:1000E000D7010008D7010008D70100080000000070
:1000F0000000000000000000000000000000000000
:1001000000000000000000000000000000000000EF
:100110000000000000000000D7010008D70100081F
:1001200000F002F800F03CF80AA090E8000C8244CD
:100130008344AAF10107DA4501D100F031F8AFF2AA
:10014000090EBAE80F0013F0010F18BFFB1A43F0B5
:10015000010318474C4601006C460100103A24BFC9
:1001600078C878C1FAD8520724BF30C830C144BF1C
:1001700004680C607047000000230024002500265E
:10018000103A28BF78C1FBD8520728BF30C148BFFA
:100190000B6070471FB5AFF300801FBD10B510BDD9
:1001A00004F0A0FD1146FFF7F5FF02F04DF904F051
:1001B000BEFDFFF7F3FF04F0C1FD000009488047D2
:1001C00009480047FEE7FEE7FEE7FEE7FEE7FEE739
:1001D000FEE7FEE7FEE7FEE704480549054A064B51
:1001E000704700000D23000821010008C086002090
:1001F000C08C0020C0880020C08800202849084307
:10020000284908607047F0B50F23C47801784FF093
:10021000E0220127E4B1D2F80C4D867804F4E064C2
:10022000C4F5E064240AC4F10405E34044781E40A8
:10023000AC4026433301114481F800340078410971
:1002400000F01F0002EB81018740C1F80071F0BD92
:1002500001F01F008740480902EB8000C0F8807160
:10026000F0BD114A114001430E48001F0160704764
:100270004FF0E0220029D2F8101D01D0014300E028
:100280008143C2F8101D70474FF0E021042808692F
:1002900002D140F0040001E020F004000861704742
:1002A0000000FA050CED00E080FFFF1FC34910B508
:1002B000884202D1012144150AE0C149884202D195
:1002C0000121041504E0BF4988420AD10121CC0371
:1002D000204601F085F82046BDE81040002101F0DD
:1002E0007FB810BD30B54268B74B0C791A400B6827
:1002F00042EA0422134343608268B44B4D791A40AA
:10030000D1E9024342EA4502234313438360C26AB0
:10031000097C22F47002491EC9B242EA0151C1624D
:1003200030BD00210160017141718160C160012116
:10033000017470470029816802D041F0010101E099
:1003400021F00101816070470029816802D041F4E9
:10035000807101E021F4807181607047002A426859
:10036000C9B201D00A4300E08A4342607047816805
:1003700041F0080181607047014689680020090743
:1003800000D501207047816841F004018160704709
:10039000014689680020490700D5012070470029DF
:1003A000816802D041F4A00101E021F4A001816044
:1003B0007047014689680020490200D50120704736
:1003C0004268491E22F4604242EA4131416070476E
:1003D0000029416802D041F4006101E021F400618C
:1003E0004160704770B5072609290AD9C568A1F18F
:1003F0000A0404EB4404A640B543A3401D43C56072
:1004000007E0056901EB4104A640B543A3401D4345
:1004100005611F23072A09D2446B521E02EB820298
:1004200093409C4391400C43446370BD0D2A09D214
:10043000046BD21F02EB820293409C4391400C4319
:10044000046370BDC46A0D3A02EB820293409C4380
:1004500091400C43C46270BD0029816802D041F410
:10046000801101E021F4801181607047C06C80B27E
:10047000704752484C30006870470029416802D0EC
:1004800041F4806101E021F48061416070470029FE
:10049000416802D041F4805101E021F48051416073
:1004A0007047826822F4E0420A4382607047002964
:1004B000816802D041F4004101E021F400418160F3
:1004C00070470029816802D041F4021101E021F453
:1004D000021181607047014689680020890200D5B9
:1004E0000120704770B5072609290AD9C568A1F10E
:1004F0000A0404EB4404A640B543A3401D43C56071
:1005000007E0056901EB4104A640B543A3401D4344
:100510000561836BC3F30154121B921C02EB820230
:100520001F249440A34391400B43836370BD826BAF
:10053000491E22F4401242EA015181637047425041
:1005400070470844806A80B270474268204B1A4066
:100550000A4342607047416282627047426822F0FB
:100560001F020A43426070471A490028D1F8080464
:1005700002D040F4000001E020F40000C1F80804BB
:1005800070470246126800200A4200D001207047DE
:10059000C9430160704730B50246002054680B0A19
:1005A000CDB211682C40194202D0002C00D001209D
:1005B00030BD6FEA11210160704700000024014046
:1005C00000280140003C0140FFFEF0FFFDF7F1FF75
:1005D000FFFD3FFF0020014010B5012000F012FF99
:1005E000BDE81040002000F00DBF1C4908607047B6
:1005F0001A49091F0860704718498431086070471C
:10060000174A118821F46071014311807047144A20
:10061000118821F07F01014311807047104A2C3A64
:10062000115070470E492C39085A70470B489C30BE
:100630000068C0B270470A480830018841F00101E3
:10064000018070470548A0300068C0B27047044878
:100650000830018841F002010180704704860D4294
:100660002C6C004010B501214C07204600F0C1FE63
:100670002046BDE81040002100F0BBBE70B5374CED
:10068000226840F6FE738340D1E901659A430B6806
:10069000C96833430D432B4383401343236070BD2C
:1006A0000021016041608160C16070472C4B0122D4
:1006B0008240D3F8000409B1104300E09043C3F82E
:1006C00000047047264B9A148240D3F8000409B105
:1006D000104300E09043C3F8000470470209012072
:1006E0001F4B90400029D3F8041401D0014300E0CF
:1006F0008143C3F80414704719490028D1F8040451
:1007000002D040F0030001E020F00300C1F804042F
:100710007047134B8140D3F800040AB1084300E04E
:100720008843C3F8000470470C4A10448160704746
:100730000A4A104441617047082802D142EA012167
:1007400001E042EA0141054A104401627047034951
:1007500001EB9000C06A80B2704700000074004056
:100760000070004002684FF6FE7300211A400260DC
:10077000016041608160C1606949694A08399042FD
:1007800003D1486840F00F0006E0654A14329042F9
:1007900004D1486840F0F00048607047604A283251
:1007A000904203D1486840F47060F5E75C4A3C32FF
:1007B000904203D1486840F47040EDE7584A503207
:1007C000904203D1486840F47020E5E7544A64320F
:1007D000904203D1486840F47000DDE7504A783217
:1007E000904203D1486840F07060D5E74D4A90428E
:1007F00004D1D1F8040440F00F0007E0494A143254
:10080000904206D1D1F8040440F0F000C1F804048D
:100810007047444A2832904204D1D1F8040440F48D
:100820007060F3E73F4A3C32904204D1D1F80404AF
:1008300040F47040EAE73B4A50329042E8D1D1F8A8
:10084000040440F47020E1E770B5026847F6F073E5
:100850009A430D6A8B680C692B43D1E905653443D3
:100860002343CC692B432343D1E909542B4323432E
:1008700013430360CA6842600A6882604968C160C5
:1008800070BD0021016041608160C1600161416112
:100890008161C16101624162816270470029016822
:1008A00002D041F0010102E04FF6FE7211400160FA
:1008B0007047002A026801D00A4300E08A430260C0
:1008C000704741607047406880B270470246002020
:1008D0001549D30002D5D1F8001400E0096811428F
:1008E00000D0012070471049C20002D5C1F80404AD
:1008F000704748607047024600200B49D30002D57C
:10090000D1F8001400E00968114200D001207047BE
:100910000549C20002D5C1F8040470474860704719
:100920000800024008040240000002403448002150
:10093000016041608160C16032494161704730B5FA
:100940002F4A8179036859B311460C689C430C60A7
:100950004B680468A3434B600479A3181C680568BE
:100960002C431C608B680468A3438B60CB680468CD
:10097000A343CB604379A1F58061102B0AD101F527
:1009800081610A6803681A430A604A680068024382
:100990004A6030BD99180A68006802430A6030BD99
:1009A0000079104401689943016030BD0021016065
:1009B00001710C22427181717047114910310A682E
:1009C00002430A60704702460D490020143109684D
:1009D000114200D001207047094914310860704766
:1009E000074B01461A6800205B690A400B4202D09F
:1009F000002A00D001207047014914310860704777
:100A000000040140FFFF0F00FC4A116801F03801AB
:100A1000014311607047F9490A6822F008020A6030
:100A20000A6802430A607047F4490A6822F010021B
:100A30000A600A6802430A607047F048F049416062
:100A4000F04941607047ED48ED494160ED49416032
:100A50007047EA48016941F0800101617047E74849
:100A6000016941F0800101617047E4490420CA68CE
:100A7000D20701D001207047CA68520701D5022071
:100A80007047C968C906FBD50320704700B5034607
:100A9000FFF7EBFF03E000BFFFF7E7FF5B1E012856
:100AA00002D1002BF8D101E0002B00D1052000BDC0
:100AB00070B505464FF430263046FFF7E7FF0428AF
:100AC00011D1CE4C206940F002002061656120699F
:100AD00040F0400020613046FFF7D8FF216941F621
:100AE000FD721140216170BD30B54FF430252846AC
:100AF000FFF7CCFF042810D1C04C206940F004005F
:100B00002061206940F0400020612846FFF7BEFFC9
:100B1000216941F6FB721140216130BD00B50346E9
:100B2000FFF7A3FF03E000BFFFF79FFF5B1E012855
:100B300002D1002BF8D101E0002B00D1052000BD2F
:100B400030B54FF430252846FFF7E8FF042810D1D0
:100B5000AA4C206940F004002061206940F0400068
:100B600020612846FFF7DAFF216941F6FB72114048
:100B7000216130BDA1490020C969890700D5012044
:100B8000704770B5A525FFF7F5FF00B100254FF4BC
:100B900030263046FFF77AFF042827D1974C984833
:100BA000A0609848A060206940F020002061206982
:100BB00040F0400020613046FFF768FF41F6EF76D5
:100BC00004280ED1206941F6DF71084020612069B8
:100BD00040F0100020618C4805804FF40050FFF772
:100BE00055FF052802D021693140216170BDF0B563
:100BF00005464FF4005C0E466046FFF747FF0428A9
:100C000014D17E4C206940F0010020612E806046A6
:100C1000FFF73CFF41F6FE77042804D1300C6880D2
:100C20006046FFF733FF216939402161F0BDF0B51F
:100C300005464FF400570E463846FFF727FF0428B5
:100C40000CD16E4C206940F0010020612E803846A6
:100C5000FFF71CFF2169BA1E11402161F0BDF0B5FC
:100C600005464FF400570E463846FFF70FFF04289D
:100C700013D1624C6248A0606248A060206940F0D5
:100C8000100020612E803846FFF700FF052804D0B1
:100C9000216941F6EF7211402161F0BD2DE9F04369
:100CA000C043C4B2C0F30725C0F30746070E4FF494
:100CB00000594846FFF7EAFE04283AD1DFF83CC164
:100CC0004F49CCF808104F49CCF80810DCF8101048
:100CD000DFF8388141F01001CCF81010FF2C06D05D
:100CE000A8F808484846FFF7D1FE042818D1FF2D80
:100CF00006D0A8F80A584846FFF7C8FE04280FD1C6
:100D0000FF2E06D0A8F80C684846FFF7BFFE04285F
:100D100006D1FF2F06D0A8F80E784846FFF7B6FE9A
:100D2000052806D0DCF8101041F6EF721140CCF81F
:100D30001010BDE8F08370B506464FF43025284604
:100D4000FFF7A4FE04282BD12C4C2D48A0602D4881
:100D5000A060206940F020002061206940F0400040
:100D600020612846FFF792FE41F6DF71042818D172
:100D70002069084020612169244841F01001216167
:100D80000EB1002100E0A521A0F800182846FFF7C9
:100D90007DFE052804D0216941F6EF7211402161E2
:100DA00070BD0528FCD022690A40226170BDF0B5F3
:100DB0000546124C12480E461746A0601148A06026
:100DC0004FF4005C6046FFF761FE042814D12069EF
:100DD00040F0100020613E432E430B4946F0F800DE
:100DE000891C08806046FFF751FE052804D0216960
:100DF00041F6EF7211402161F0BD00000020024079
:100E000023016745AB89EFCD00F8FF1F00F0FF1FFE
:100E10001C48C069800870471A48006A7047194921
:100E200000200968890600D501207047154A00296D
:100E3000116901D0014300E081431161704701460F
:100E40000020104A012904D1D169C90700D001202E
:100E50007047D2680A42FAD170470A49C8607047A1
:100E600008490420CA68D20701D001207047CA6827
:100E7000520701D502207047C968C906FBD5032077
:100E80007047000000200240904910B5884206D10A
:100E90000121042000F0A4FA002104203BE08C4949
:100EA000884206D10121082000F09AFA002108208A
:100EB00031E08849884206D10121102000F090FAE3
:100EC0000021102027E08449884206D101212020FA
:100ED00000F086FA002120201DE08049884206D1DA
:100EE0000121402000F07CFA0021402013E07C49E1
:100EF000884206D10121802000F072FA0021802072
:100F000009E0784988420AD184150121204600F081
:100F100067FA00212046BDE8104000F061BA10BD1C
:100F200010B50121084600F05BFA0021BDE8104031
:100F3000012000F055BAF0B5CB780022DC0603F0B2
:100F40000F0301D58C7823430C884FF00F0C14F05D
:100F5000FF0F4FF0010E1BD0D0F800600D880EFA85
:100F600002F42540A5420FD195000CFA05F726EAB8
:100F7000070703FA05F6CD783E43282D01D14461D9
:100F800002E0482D00D10461521C082AE6D3066015
:100F90000A88FF2A1ED946685FF0000202F10805A0
:100FA0000EFA05F40D882540A5420FD195000CFAE4
:100FB00005F726EA070703FA05F6CD783E43282D04
:100FC00000D14461CD78482D00D10461521C082A1B
:100FD000E4D34660F0BD4FF6FF71018002218170BD
:100FE0000421C17070470246926800200A4200D076
:100FF00001207047806880B270470246D2680020A6
:101000000A4200D001207047C06880B27047016179
:101010007047416170470AB1016170474161704793
:10102000C160704741F4803282618161826181696F
:101030008069704710B52C4B1A684FF680742240B7
:1010400042EA00100843186010BD2849C861704783
:10105000F0B5254C002801DAE36900E06368450D2E
:101060002E0185B2C0F30157B540C0F30342032FF0
:1010700006D123F07062636823F07063636008E058
:10108000C60203D503269640B34300E0AB4343F0CA
:10109000706201B12A43002801DAE261F0BD6260AA
:1010A000F0BD10B58A0721F003040F49120F214447
:1010B0000F238C6893409C438C608B689040034363
:1010C0008B6010BD0949DC310860704700080140A1
:1010D000000C0140001001400014014000180140C4
:1010E000001C01400020014000000140000020429F
:1010F00010B501210C07204600F07BF92046BDE821
:101100001040002100F075B9244908627047234956
:1011100008617047224A116821F0E0010143116023
:1011200070471E49A031086070471D4B1A6822F0B5
:10113000030202431A604FF0E020D0F8102D01297D
:1011400042F00401C0F8101D01D130BF00E020BF03
:10115000D0F8101D21F00401C0F8101D7047104890
:10116000016841F004010160026842F0020202607D
:101170000C49086840F00400086030BF7047084917
:10118000024649680020114200D0012070470449FE
:101190000A6842EA800008607047000000000E42C2
:1011A0000070004010ED00E0A448016841F001012A
:1011B00001604168A24A114041600168A14A1140A2
:1011C0000160016821F48021016042684FF41F0131
:1011D00022F4FE0242608160704798490A6822F456
:1011E00080320A600A68B0F5803F22F480220A60EB
:1011F00007D0B0F5802F03D1086840F4A020086024
:101200007047086840F48030F9E703460020590928
:101210008A4A012901D1116804E0022901D1116A29
:1012200000E0516A03F01F02012393400B4200D0FB
:101230000120704730B500244FF4A0653120FFF73E
:10124000E4FF641CAC4201D00028F7D03120FFF746
:10125000DCFF002800D0012030BD784A116821F061
:10126000F80141EAC0001060704777490860704794
:10127000724B5A68084322F47C121043586070473E
:101280007149086670476D4A516821F003010143B6
:10129000516070476948406800F00C007047674A29
:1012A000516821F0F001014351607047634A516871
:1012B00021F4E061014351607047604A516821F4B4
:1012C000605141EAC000506070475C4A0029517A81
:1012D00001D0014300E08143517270475A49D8312F
:1012E00008607047554A516821F4404101435160FC
:1012F00070475249002220310A7001F82029012844
:1013000002D0042802D1052081F8200070474F49FF
:101310000860704749490A6A02430A6270474B49AC
:1013200044390860704710B5444A5168484B11F081
:101330000C0103D0042901D0082901D0036011E079
:1013400051685368022401F4701104EB914113F4C5
:10135000803F02D053689B0301D53E4B00E03C4BDD
:101360005943016051683C4B01F0F00109095C5C94
:101370000168E1404160546804F4E064240A1C5DA3
:1013800021FA04F48460546804F46054E40A1B5D98
:10139000D940C1605268304B02F44042920B1B1F8F
:1013A0009A5CB1FBF2F1016110BD244A0029516938
:1013B00001D0014300E08143516170471F4A002979
:1013C000916901D0014300E08143916170471B4A5C
:1013D0000029D16901D0014300E08143D161704708
:1013E000164A0029D16801D0014300E08143D16051
:1013F0007047124A0029116901D0014300E081437E
:101400001161704711494039086070470E49C8643E
:1014100070470A49C87170470848416A41F08071B5
:10142000416270470549024689680020114200D098
:101430000120704701498872704700000010024087
:101440000000FFF8FFFFF6FE000042428004424227
:1014500000127A0000093D00040000203D4A0029E6
:10146000B2F8001801D0014300E08143A2F800184F
:1014700070473948018841F01001018070473648B3
:10148000018821F0100101807047334914318888A8
:10149000098840EA0140704700B50246FFF7E9FFBE
:1014A0002D48110C1430018082805DF804EBE6E7D2
:1014B00000B50246FFF7DDFF2748C2F30341001DD8
:1014C000018082805DF804EBD9E700B50246FFF7A2
:1014D000D0FF2148110C1C30018082805DF804EBA4
:1014E000CDE71D480C3001888088090740EA11309B
:1014F00070471848B0F804188906FBD5704715489E
:10150000B0F8041821F00801A0F80418B0F8041885
:101510000907FBD57047104902460988002011428F
:1015200000D0012070470C4A118881431180704718
:101530000949091F8B880A880340D9B2024202D0A8
:1015400009B10120704700207047034A1188814388
:10155000118070470020004004280040FA4910B56F
:10156000884202D10121C41486E0B0F1804F06D137
:1015700001210846FFF73DFF0021012067E0F34904
:10158000884206D101210220FFF733FF002102200B
:101590005DE0EF49884206D101210420FFF729FFD1
:1015A0000021042053E0EB49884206D101210820A4
:1015B000FFF71FFF0021082049E0E749884206D1D4
:1015C00001211020FFF715FF002110203FE0E34923
:1015D000884206D101212020FFF70BFF00212020A7
:1015E00035E0DF49884202D10121441444E0DD495D
:1015F000884202D10121CC043EE0DB49884202D17D
:1016000001210C0538E0D949884202D101214C055D
:1016100032E0D749884206D101214020FFF7E9FE98
:101620000021402013E0D349884206D101218020C7
:10163000FFF7DFFE0021802009E0CF4988420AD170
:10164000841501212046FFF7D4FE00212046BDE885
:101650001040FFF7CEBEC949884202D101210C04D7
:101660000AE0C749884202D101214C0404E0C5497F
:1016700088420AD101218C042046FFF7B1FE2046A2
:10168000BDE810400021FFF7ABBE10BD30B50288A9
:10169000AD4CB34DA0420DD0A8420BD0B0F1804F5D
:1016A00008D0AA4B984205D0A94B984202D0A94B2A
:1016B000984203D122F070034A881A43A64B9842FD
:1016C00006D0A64B984203D022F44073CA881A432E
:1016D00002808A88A04282850A8802850AD0A842B0
:1016E00008D0A64A904205D0A54A904202D0A54A09
:1016F000904201D1097A01860121818230BDF0B585
:10170000028C22F001020284048C8288038B24F074
:10171000020523F073060B880C8933434E888A4FE9
:101720002C432643B8420BD08D4CA04208D0934C9A
:10173000A04205D0924CA04202D0924CA0420DD1C2
:1017400026F008044D898E88254325F004052E4394
:1017500022F440748D89CA8925432A4382800383F9
:10176000C98881860684F0BD30B5028C22F0100253
:101770000284028C8388048B22F0200224F4E64544
:101780000C88240645EA14440D892D0542EA1545C6
:101790004A88120545EA12426B4DA84202D0704DAC
:1017A000A84215D14D8922F080022D0542EA154547
:1017B0008A8825F04005120545EA12428D8923F4F6
:1017C0004063AD0443EA1545CB899B0445EA1343C6
:1017D00083800483C9880187028430BD70B5028C80
:1017E00022F480720284028C8388848B0E8924F018
:1017F00073050C8822F400722C43350642EA154525
:101800004A88120645EA12424F4DA84202D0544D72
:10181000A84215D14D8922F400622D0642EA1545F1
:101820008A8825F48065120645EA12428D8923F4E0
:1018300040532D0543EA1545CB891B0545EA134363
:1018400083808483C9888187028470BD30B5028C0F
:1018500022F480520284038C8288848B24F4E6452F
:101860000C88240645EA144423F400550B891B0711
:1018700045EA13434D882D0743EA1545324B9842FC
:1018800002D0374B984205D122F480438A899205D1
:1018900043EA124282808483C988A0F840100584FC
:1018A00030BD828B22F440628283828B42EA012225
:1018B00082837047828B22F00C028283828B0A43E0
:1018C00082837047028B22F440620283028B42EAD9
:1018D00001220283704770B5048C24F01004048444
:1018E000068B048C26F473461B0746EA1343120644
:1018F00043EA12420D05144B2D0C98420ED0184BA2
:1019000098420BD0B0F1804F08D0104B984205D0D0
:101910000F4B984202D00F4B984205D124F0200182
:10192000294341F0100104E024F0A0030B4343F0ED
:1019300010010283018470BD028B22F00C0202832D
:10194000028B0A4302837047002C014000040040D0
:1019500000080040000C004000100040001400404F
:1019600000340140004C014000500140005401404F
:1019700000180040001C00400020004000400140D2
:10198000004401400048014030B5048C24F00104BB
:101990000484058B048C1B0542EA134325F0F305F0
:1019A000F94A2B4390420ED0F84A90420BD0B0F146
:1019B000804F08D0F64A904205D0F64A904202D0B5
:1019C000F54A904202D124F0020201E024F00A021A
:1019D0000A4342F001010383018430BD2DE9F05F29
:1019E000E94EEA4FDFF8A883DFF8A893DFF8A8B341
:1019F00004460D464FF0804AB04206D0BC4204D0A7
:101A0000544502D0444500D0484628886988AA88B1
:101A10002B8938B92046FFF7B7FFE9882046BDE893
:101A2000F05F89E7042807D12046FFF754FFE988D3
:101A30002046BDE8F05F45E70828208C2CD120F433
:101A400080702084A08BB4F820C01B0520F0F30028
:101A500042EA13434FEA016E03434FEA1E4EB4427B
:101A600009D0BC4207D0544505D0444503D04C456D
:101A700001D05C4504D12CF4007040EA0E0002E075
:101A80002CF42060084340F48070A3832084E9880C
:101A90002046BDE8F05F0DE720F480502084B4F8C4
:101AA0001CC0208C12062CF4734C1B074FEA017EDD
:101AB0004CEA12424FEA1E4E42EA1343B44209D0A6
:101AC000BC4207D0544505D0444503D04C4501D015
:101AD0005C4504D120F4005040EA0E0002E020F4FE
:101AE0000240084340F48050A3832084E9882046C4
:101AF000BDE8F05FD5E62DE9F0410C4600254988A8
:101B00000746012601B90225A288012A00D1022632
:101B1000208823890028384610D1FFF735FFE18857
:101B20003846FFF709FF2389324629463846FFF732
:101B3000D2FEE1883846BDE8F041C3E6FFF7CBFEB0
:101B4000E1883846FFF7BEFE2389324629463846EB
:101B5000FFF71AFFE1883846BDE8F041ECE630B502
:101B60000A884C888B88CD8822432B431A430C89E2
:101B70004B89224389891A430A43A0F8442030BD87
:101B80004FF6FF71818000210180C1804180017288
:101B9000D9E60021018041808180C180018141819D
:101BA0008181C181CFE600210180418001228280B4
:101BB000C1800181C7E60021018041808180C18010
:101BC000018141818181BEE60029018802D041F076
:101BD000010101E021F001010180B4E6002930F8A3
:101BE000441F02D041F4004101E0C1F30E01018025
:101BF000A9E6002A828901D00A4300E08A43828153
:101C0000A1E681829FE61143A0F848109BE6002AD6
:101C1000828901D00A4300E08A43828193E60189E8
:101C200021F0070101818EE6028922F070020A4349
:101C3000028188E6028922F070020A43028101894A
:101C400041F0070101817EE670B50D46114604465C
:101C5000602D4FF0010202D1FFF73DFE01E0FFF7DA
:101C600093FE208920F0700028432081208940F0D5
:101C70000700208170BD10B5048942EA0323E4B255
:101C80000B432343038110BD10B50446FFF7F3FF58
:101C9000208940F07700208110BD10B50446FFF781
:101CA000EAFF208940F48040208110BD01858282B6
:101CB00049E6028822F070020A43028043E670B5CA
:101CC0000689058B048C26F007060E434FF6FC416F
:101CD0000D4040F201110D4324F0220442EA0311A9
:101CE000214306810583018470BD028B22F07002BE
:101CF0000A43028327E6028B22F4E04242EA0121F2
:101D0000018320E6828B22F070020A4382831AE666
:101D1000828B22F4E04242EA0121818313E600290A
:101D2000018802D041F0800101E021F080010180B2
:101D300009E60029818802D041F0040101E021F088
:101D400004018180FFE50029818802D041F008016B
:101D500001E021F008018180F5E50029818802D0A9
:101D600041F0010101E021F001018180EBE5028BEE
:101D700022F008020A430283E5E5028B22F40062A6
:101D800042EA01210183DEE5002C014000340140DC
:101D90000004004000080040000C0040828B22F04C
:101DA00008020A438283CEE5828B22F4006242EA73
:101DB00001218183C7E5028B22F004020A430283DA
:101DC000C1E5028B22F4806242EA01210183BAE577
:101DD000828B22F004020A438283B4E5828B22F4D0
:101DE000806242EA01218183ADE5028B22F080020C
:101DF0000A430283A7E5028BC2F30E0242EA0121E5
:101E00000183A0E5828B22F080020A4382839AE557
:101E1000828BC2F30E0242EA0121818393E5028C98
:101E200022F002020A4302848DE5028C22F00802AD
:101E30000A43028487E5028C22F0200242EA011163
:101E4000018480E5028C22F0800242EA01110184C3
:101E500079E5028C22F4007242EA0121018472E5E4
:101E6000028C22F4006242EA012101846BE5028CBB
:101E700022F4005242EA0131018464E510B50123E5
:101E8000048C8B409C430484038C8A40134303845A
:101E900010BD10B50423048C8B409C430484038C38
:101EA0008A401343038410BD30B50124058C00F132
:101EB00018038C40A543058409B1082907D103EB19
:101EC0005100016821F07001016001680AE0091FFA
:101ED00088B203EB5000016821F4E0410160016821
:101EE0001206120C1143016030BD0029018802D096
:101EF00041F0020101E021F00201018023E5002907
:101F0000018802D041F0040101E021F004010180C8
:101F100019E50029818802D041F0800101E021F01B
:101F2000800181800FE5028822F008020280028889
:101F30000A43028007E5828822F07002828082884C
:101F40000A438280FFE4028922F0070202810289AB
:101F50000A430281F7E4028922F0800202810289A9
:101F60000A430281EFE48184EDE48185EBE481861C
:101F7000E9E40187E7E48187E5E4A0F84010E2E4C2
:101F8000028822F44072028002880A430280DAE466
:101F9000808ED8E4008FD6E4808FD4E4B0F840007F
:101FA000D1E4808CCFE4008DCDE40246128A00207B
:101FB0000A4200D00120C6E4C9430182C3E40246BC
:101FC000138A002092890B4202EA010202D0002A01
:101FD00000D00120B7E4C9430182B4E4C64910B57A
:101FE00088420AD101218C032046FFF7F9F92046E7
:101FF000BDE810400021FFF7F3B9C049884202D183
:1020000001214C0410E0BE49884202D101218C0418
:102010000AE0BC49884202D10121CC0404E0BA495B
:1020200088420AD101210C052046FFF7E2F920463B
:10203000BDE810400021FFF7DCB910BD30B5044603
:10204000008A85B00D464CF6FF710840E9880143CF
:102050002182A0894EF6F3110840A9882A891143EC
:102060006A8902431143A181A08A4FF6FF410840CB
:10207000A9890143A1826846FFF755F99E48844229
:1020800001D1039800E00298A1890904002900EB1E
:10209000C00101EB0010296802DA4FEA410101E0BA
:1020A0004FEA8101B0FBF1F06422B0FBF2F14FEA9C
:1020B00001114FEA11136FF018056B43A58900EB6E
:1020C000830032232D0406D503EBC000B0FBF2F0F1
:1020D00000F0070005E003EB0010B0FBF2F000F0A9
:1020E0000F000843208105B030BD4FF41651016048
:1020F00000218180C18001810C2242818181704751
:1021000030B5028A4FF2FF031A400B884D888C8845
:10211000C9882B430C4323431343038230BD002162
:10212000018041808180C18070470029818902D06F
:1021300041F4005101E021F400518181704710B554
:10214000C1F3421301F01F040121A140012B01D171
:102150000C3004E0022B01D1103000E01430002AD2
:10216000026801D00A4300E08A43026010BD002AE1
:10217000828A01D00A4300E08A4382827047028A41
:1021800022F00F020282028A0A4302827047828989
:1021900022F40062828182890A4382817047002989
:1021A000818902D041F0020101E021F00201818128
:1021B0007047028A22F020020282028A0A430282C7
:1021C00070470029018A02D041F4804101E021F4E6
:1021D000804101827047C1F3080181807047808887
:1021E000C0F308007047818941F001018181704787
:1021F000028BD2B20283028B42EA01210183704733
:10220000028B02F47F420283028B0A4302837047EF
:102210000029818A02D041F0200101E021F0200153
:10222000818270470029818A02D041F0100101E0CB
:1022300021F01001818270470029818A02D041F08B
:10224000080101E021F0080181827047002981899D
:1022500002D041F4004101E0C1F30E0181817047D9
:102260000029818A02D041F4006101E021F400617B
:1022700081827047828A22F004028282828A0A4323
:10228000828270470029818A02D041F0020101E078
:1022900021F00201818270470246128800200A4222
:1022A00000D001207047C9430180704770B501F02C
:1022B0001F0601250024C1F3421305FA06F2012B83
:1022C00001D1838904E0022B01D1038A00E0838AD3
:1022D0004FEA11210088134205FA01F500EA0500D2
:1022E00001D000B10124204670BD0A0A01219140AD
:1022F000C94301807047000000380140004400409D
:1023000000480040004C00400050004010B54648D6
:10231000016841F0010101604168444A1140416097
:102320000168434A11400160016821F48021016085
:10233000416821F4FE0141604FF41F01816000F00B
:102340002FF83C494FF00060086010BD10B5364AC8
:102350005068394B10F00C01384803D0042901D0E3
:10236000082901D0036011E051685368022401F488
:10237000701104EB914113F4803F02D053689B032A
:1023800001D52F4B00E02C4B5943016052682B497B
:10239000C2F30312091D895C0268CA40026010BDC5
:1023A000214900200A6842F480320A604FF4A06399
:1023B0000A68401C12F4003F01D19842F8D1086825
:1023C000800330D51F48026842F0100202600268A4
:1023D00022F003020260026842F0020202604868D2
:1023E000486048684860486840F4806048604868D1
:1023F00020F47C104860486840F4E81048600868A1
:1024000040F08070086008688001FCD5486820F0C2
:1024100003004860486840F0020048604868C0F324
:1024200081000228FAD17047001002400000FFF836
:10243000FFFFF6FE08ED00E000127A001400002015
:1024400000093D00002002402DE9F05F24490A20E8
:10245000087000F035FD02F038FA00F069FE00F077
:10246000F2FD01F0E1FC01F031FE00F00AFA02F0A9
:1024700053FB012000F038FA194C0126194FDFF800
:102480006880DFF868900025DFF864B04EF6602AB7
:10249000A41C00BFC7F8A46102F067F90FF055FE55
:1024A00002F002F898F8000008B100F0A2FED9F896
:1024B00000010028208808D108B900F0C4FD208858
:1024C0005045E7D8401C2080E4E76428E2D3ABF80D
:1024D000A05000F07AFD002000F006FA2580D9E730
:1024E0002800002000802142FA0000200000214244
:1024F0000010002042F6E06305E019460A00A1F151
:10250000010189B2FAD10100A0F1010080B2F4D139
:102510007047F0B5ED49DFF8B8C301EB40010A465A
:1025200001F5905102F58052CCE902120E88E94D76
:1025300000F5C061138801F00704E74F2A5D07EB3F
:10254000D101B3421DD20B7800F56050134200F068
:10255000070207EBD00003D00178AA5C11430EE01C
:10256000DE4E345D23400B700178AB5C194207D01E
:10257000DCF80C30002119800178B25C1140017048
:10258000F0BD087810430870F0BDD04970B501EB7C
:10259000400101F59053CE4A01F58051C2E9023164
:1025A00000F5C0610C46CC4B04F00706CB4C03EBA6
:1025B000D1010D78A65D35400D7000F5B0510D4686
:1025C00003EBD10105F007050E78655D00F560505D
:1025D0002E400E7003EBD00100F007000B78205C5A
:1025E00003400B70916800200880D168088070BD9E
:1025F000F0B5DFF8D8C2B84EB64DB54F002000BFD9
:102600000CEB400101F5905201F5805100F5B054FA
:10261000C7E9022106EBD40304F007041B782C5D04
:1026200023420FD00B88128893420BD200F5C06270
:1026300006EBD20402F007022478AA5C144201D10E
:102640005B1C0B80401C80B2C828D9D3F0BDF0B50C
:10265000DFF878C2A04E9F4D9D4FC8200CEB400183
:1026600001F5905201F5805100F5B054C7E90221FF
:1026700006EBD40304F007041B782C5D23420FD033
:102680000B88128893420BD200F5C06206EBD2048D
:1026900002F007022478AA5C144201D15B1C0B8073
:1026A000401C80B2F628D9D3F0BDF0B5DFF81CC2CB
:1026B000894E884D864FF6200CEB400101F5905273
:1026C00001F5805100F5B054C7E9022106EBD403AF
:1026D00004F007041B782C5D23420FD00B8812886E
:1026E00093420BD200F5C06206EBD20402F007025F
:1026F0002478AA5C144201D15B1C0B80401C80B280
:10270000FA28D9D3F0BDF0B5DFF8C0C1724E714DD3
:102710006F4FFA200CEB400101F5905201F580510A
:1027200000F5B054C7E9022106EBD40304F0070416
:102730001B782C5D23420FD00B88128893420BD25A
:1027400000F5C06206EBD20402F007022478AA5C0E
:10275000144201D15B1C0B80401C80B2FF28D9D9E8
:10276000F0BD2DE9F04700254FF080400582584F1D
:10277000B8880A30B8803878401C387000F028FAE1
:102780003878554C534E632808D93D7094F8E101D0
:102790003179084384F8E101FFF787FF38784FF07B
:1027A0000A09B0FBF9F2B84609FB12004B4F0728A3
:1027B00007D1FFF74CFF94F8E101F978084084F85D
:1027C000E10198F800004346B0FBF9F209FB120161
:1027D000022905D194F8E111F278114384F8E1114E
:1027E0009846322807D1FFF703FF94F8E1013979C1
:1027F000084084F8E10198F800005A280AD1FFF750
:1028000082FFB8F80200401CA8F8020034480570A6
:102810003448057098F8000000F00F00022803D13A
:1028200002F0E1F802F07FF9B8F80200C446B0FB0C
:10283000F9F209FB1201052905D194F8E1217B7910
:102840001A4084F8E12129B994F8E1117279114311
:1028500084F8E111B0F5967F04D194F8E101B979DB
:10286000084004E038B994F8E101B179084384F8EC
:10287000E101BDE8F087B0F5167FFAD3ACF802505D
:10288000F7E73EB501210846FEF7A1FD48F6A04056
:10289000ADF804000120ADF800000020ADF80600FE
:1028A000ADF802004FF0804469462046FEF7EEFE88
:1028B00001212046FFF78FFB012211462046FFF73A
:1028C00098F901212046FFF77FF93EBD0010002056
:1028D000E0000020EC5F000800100020F45F00081A
:1028E0000C0100200D0100202DE9F84304460021D1
:1028F0004FF00060FDF7B5FC4FF48060FDF77EFC03
:1029000025208DF8000002268DF8016000258DF845
:1029100002508DF803406846FDF775FC0E208DF8D7
:1029200000004FF003088DF801808DF80260012649
:102930008DF803606846FDF766FC27208DF80000DF
:102940008DF801608DF802508DF803406846FDF760
:102950005AFC1D208DF8000005208DF801008DF82F
:1029600002508DF803406846FDF74DFC1E208DF89F
:10297000000004278DF801708DF802508DF8034097
:102980006846FDF740FC32208DF8000006208DF8E7
:1029900001008DF802508DF803406846FDF733FCC6
:1029A0002E208DF800008DF801508DF802608DF812
:1029B00003606846FDF727FC1C208DF800008DF8A9
:1029C00001508DF802508DF803406846FDF71BFC5E
:1029D00028208DF800008DF801708DF802508DF8D8
:1029E00003406846FDF70FFC17208DF800008DF8B6
:1029F00001808DF802508DF803406846FDF703FC16
:102A0000BDE8F8831CB50F210020FEF74AFB4FF408
:102A10008050009000208DF804000C208DF80500F7
:102A200001208DF806006846FDF789FF4FF400602D
:102A300000906846FDF783FF1CBD1CB509210220EC
:102A4000FEF72FFB4FF40070009000208DF804007B
:102A50000C208DF8050001208DF806006846FDF772
:102A60006EFF08210220FEF71CFB4FF480700090DF
:102A70006846FDF764FF07210220FEF712FB802065
:102A800000906846FDF75BFF06210220FEF709FB78
:102A9000402000906846FDF752FF1CBD38B501216B
:102AA000F848FEF7D5FA0120ADF8000004258DF8AE
:102AB000035002248DF802406946F348FEF73BFAC2
:102AC0002003ADF800008DF80350F04D8DF8024062
:102AD00069462846FEF72FFA4FF44070ADF8000023
:102AE00014208DF803008DF802406946E848FEF78F
:102AF00022FA4FF4E070ADF8000010208DF80300CA
:102B000003208DF8020069462846FEF714FA38BD06
:102B100038B50121DB48FEF79BFACE20ADF8000066
:102B200004258DF8035002248DF802406946D648EA
:102B3000FEF701FA4FF20300ADF800008DF80350E4
:102B40008DF802406946D248FEF7F5F93020ADF81D
:102B500000008DF803508DF802406946CB48FEF71F
:102B6000EAF938BD38B50121C648FEF771FA4FF4CD
:102B70001940ADF8000001258DF8025010248DF8A1
:102B800003406946C048FEF7D6F9F820ADF80000CA
:102B90008DF802508DF803406946BD48FEF7CBF929
:102BA0004FF4F050ADF800008DF802508DF803405E
:102BB0006946B648FEF7BFF90420ADF800008DF86D
:102BC00002508DF803406946B248FEF7B4F938BDAB
:102BD00070B5B14ED6F80451B149B0480B7890F8B1
:102BE0008040B04900221DB10A7024F0010408E0C1
:102BF00091F900509D4202DA6D1C0D7003E044F023
:102C0000010480F88040D6F808412CB14A7090F851
:102C1000804024F002040AE091F901409C4202DA6B
:102C2000641C4C7005E090F8804044F0020480F889
:102C30008040D6F80C412CB18A7090F8804024F086
:102C400004040AE091F902409C4202DA641C8C7090
:102C500005E090F8804044F0040480F88040D6F805
:102C600018412CB1CA7090F8804024F008040AE0A2
:102C700091F903409C4202DA641CCC7005E090F8A4
:102C8000804044F0080480F88040D6F81C412CB104
:102C90000A7190F8804024F010040AE091F9044091
:102CA0009C4202DA641C0C7105E090F8804044F00C
:102CB000100480F880407C4DD5F810412CB14A7149
:102CC00090F8804024F020040AE091F905409C42ED
:102CD00002DA641C4C7105E090F8804044F0200456
:102CE00080F88040D5F814412CB18A7190F880406A
:102CF00024F040040AE091F906409C4202DA641C88
:102D00008C7105E090F8804044F0400480F88040E9
:102D1000664ED6F800412CB1CA7190F8803023F08D
:102D200080030AE091F907409C4202DA641CCC71EE
:102D300005E090F8803043F0800380F88030D6F8CA
:102D40000451564B93F88140B3F8283E1DB10A72E6
:102D500024F0010408E091F908509D4202DA6D1C4C
:102D60000D7203E044F0010480F88140D6F8304150
:102D70002CB14A7290F8814024F002040AE091F9E3
:102D800009409C4202DA641C4C7205E090F88140D4
:102D900044F0020480F88140D6F834412CB18A72A4
:102DA00090F8814024F004040AE091F90A409C4222
:102DB00002DA641C8C7205E090F8814044F004044F
:102DC00080F88140D6F838412CB1CA7290F8814021
:102DD00024F008040AE091F90B409C4202DA641CDA
:102DE000CC7205E090F8814044F0080480F88140FE
:102DF000D6F83C412CB10A7310F8811F21F0100164
:102E00000AE091F90C209A4202DA521C0A7370BD52
:102E100010F8811F41F01001017070BD1F4B10B5FB
:102E2000A03318782249C0F300020A60214AC0F397
:102E300040041460C0F38004D460C0F3C004146183
:102E4000C0F30014D461C0F340124A60C0F3801292
:102E50008A60C009C86058781749C0F30002C1F8F9
:102E600088211649C0F340020A60C0F380024A601C
:102E7000C0F3C0028A60C0F30012CA60C0F3401001
:102E8000086110BD00023000000801400010014040
:102E9000000C0140001401400000214200100020FD
:102EA000F0000020AC0700200000224200802142F8
:102EB000A4012242A0012142008022428C812142B1
:102EC00010B501213C20FEF779FA01210846FEF7F2
:102ED00075FA064901200860FFF744FEFFF79EFFE0
:102EE000FFF716FEBDE81040D8E50000A48121429E
:102EF00010B50E48002404800D48D0F824210D4957
:102F0000C0F8A4412AB1B1F8180F401CA1F8180F5D
:102F1000FFE7B1F8F201800707D50448002201213C
:102F20001038FEF766FE0448047010BD100400401F
:102F30000000224200100020F100002028B1764A53
:102F4000764B1178DB79194311707549A1F87E0E23
:102F500070472DE9F04105460C281BD2FDF76DFDA9
:102F6000704E06EBC520FDF7A3FD00246E4FED0269
:102F70004FF4806805EB4400304480B237F81410F9
:102F8000FDF755FE641CA4B24445F3D3BDE8F041FF
:102F9000FDF75FBDBDE8F08170B50C2814D20021AB
:102FA000624B614DC4024FF4806600BF04EB4100E8
:102FB00080B21A5C1844407802EB002025F811001A
:102FC000491C89B2B142F1D370BD30B4544B564A5A
:102FD000002041F2F41141F2B63500BF33F8114040
:102FE00022F81040401C491C89B280B2A942F5D396
:102FF00040F2645140F2965533F8114022F81040E7
:10300000401C491C89B280B2A942F5D340F6640144
:1030100040F6960533F8114022F81040401C491C38
:1030200089B280B2A942F5D35FF0200133F8114094
:1030300022F81040401C491C89B280B24029F5D3C7
:1030400030BC0A2085E730B500240A20FFF7A4FF32
:10305000354A334941F2F41041F2B63532F81430B2
:1030600021F81030641C401C80B2A4B2A842F5D3F1
:1030700040F2645040F2965532F8143021F8103086
:10308000641C401C80B2A4B2A842F5D340F6640090
:1030900040F6960532F8143021F81030641C401CBC
:1030A00080B2A4B2A842F5D35FF0200032F8143009
:1030B00021F81030641C401C80B2A4B24028F5D323
:1030C00030BD174A4FF480504FF43D53002100BFEC
:1030D00022F81010401C80B29842F9D34FF4A0603F
:1030E0004FF4C06322F81010401C80B29842F9D30C
:1030F0004FF400604FF4106322F81010401C80B2AF
:103100009842F9D35FF0000022F81010401C80B202
:103110008028F9D370470000E7110020EC5F000819
:103120000010002000600008886E00200060000889
:1031300030B5F94852238381F84AF94C002000BF8A
:1031400032F8105000F5E061401C80B224F81150B4
:103150007E28F5D3F34AF448D15C01801A445278B2
:1031600089B242EA01210180F04809230370EA494B
:10317000C82010310870487030BD2DE9F041054677
:10318000112821D2FDF759FCE94E06EBC520FDF7C9
:103190008FFC0024E74FED024FF4806807EB8402B8
:1031A00037F82410528805EB4400304401EB02212B
:1031B00080B289B2FDF73BFD641CA4B24445EDD357
:1031C000BDE8F041FDF745BCBDE8F08130B5112800
:1031D0000ED2D44BD74C00214FF4006501EBC02236
:1031E00092B29A5C24F81120491C89B2A942F5D305
:1031F00030BDC9490878002809D0002008708871BE
:10320000CD4849898164416C41F0010141647047B6
:103210002DE9F04100260546012827D10020FFF7BF
:10322000D5FFC4490F20A1F8B800A1F8BA605E200C
:103230004FF6FF724FF4006321F81020401C80B25B
:103240009842F9D3FDF7F9FBBC48FDF731FC0020AB
:10325000FFF793FFB64F012407EBC420FDF728FCCE
:10326000641CA4B20A2CF7D3FDF7F3FBB44A022D79
:1032700007D1101447F67E638654801C80B29842B2
:10328000FAD3032D05D100208654801C80B2BE28BD
:10329000FAD3AC49062048709F490120488193E742
:1032A00010B59D4B02461C890020D21C0321641ED0
:1032B00006E000BF12F8013B491C1844C0B289B2B5
:1032C000A142F7DB10BDF0B5934904200D899E4B58
:1032D0009E4C9C4EAD1E0BE01F18195C7F78615C04
:1032E00006EB5002E75D801C07EB0111117080B204
:1032F000A842F1DBF0BD9349874AC878897801EB91
:103300000020908170478F49834AC878097901EB82
:103310000020D0817047F8B580498A4F31F81000FD
:10332000009002207870DFF8F0C10022104601F50D
:103330000075EE469CF8056013E000BF1EF80030F3
:1033400005EB13110C7807EB40018C7003F00F03B1
:10335000EB5CCB70C978E3B219441144401CCAB28B
:1033600080B2B042EAD3032107EB40039970D21C2C
:10337000D1B205EB1112127801F00F01DA70695C1D
:103380001971042101EB4000ACF80A00F8BDA0F56A
:103390008041B1F57A5F02D2A0F5005032E0A0F58D
:1033A00020717C2904D9A0F51072C031162A01D8E9
:1033B00088B27047A0F5C073162B01D8E03821E021
:1033C000A0F500731F2B02D8A0F5A0701AE0A0F59D
:1033D000A0631F2B01D890B27047A0F5F0721F2A8E
:1033E00001D820380EE0BF2802D800F5807009E02F
:1033F000A0F1C002BF2A02D800F5886002E01F29B0
:10340000EAD8203080B270474FF4C062904202D2B6
:1034100000F5006035E0A0F5C061914202D200F5F0
:1034200008502EE0A0F54061B72902D8A0F5E06071
:1034300027E0A0F590521346A0F56061BF2A01D89D
:1034400088B27047A0F5A052B2F57A7F01D290B24F
:103450007047A0F52052FF2A01D898B27047A0F516
:103460008052FF2A02D8A0F520600AE0FF2902D886
:1034700000F5807005E0A0F57061FF29EED8A0F599
:10348000807080B270472DE9F04302212D48DFF8AB
:10349000BC80002641703446A8F114081E4F8146B6
:1034A00021E0B889204480B2FFF771FFDFF890C0B7
:1034B00009EB440510F80C0008EB10100078A87018
:1034C000B889204480B2FFF762FF10F80C00641C3A
:1034D00000F00F0018F80000E870A878E978A4B2AE
:1034E00008443044C6B278798442DAD3032109EB28
:1034F00044008170F61CF1B208EB11131B7801F047
:103500000F01C37018F801100171042000EB440092
:103510007881BDE8F0830000F4000020BA41010882
:10352000001000200060000800500020E011002082
:1035300000600008886E002000000240006800085B
:10354000001000208C7E002080800020CE430108E7
:10355000F0B5FD4D0422A978E87802EB0121FB4E7D
:103560000844B0810024FA4F09E0B089204480B2B9
:10357000FFF70DFF29194979641CC155A4B2707970
:103580008442F2D30620687001207081F0BD30B50E
:10359000ED4CE078A17800EB012080B2FFF734FF1A
:1035A000EB4901EBD005E078A17800EB012080B277
:1035B000FFF72AFFE74900F00700085C2978084375
:1035C000287006206070E1490120488130BD30B587
:1035D000DD4CE078A17800EB012080B2FFF714FF0A
:1035E000DB4901EBD005E078A17800EB012080B247
:1035F000FFF70AFFD84900F00700085C2978084067
:10360000287006206070D1490120488130BDCE4825
:10361000CE49C278807802EB002080B28881A0F584
:103620006060023803D0C82803D1652000E0012083
:1036300071E628E730B5C54DA889A0F5606123394A
:103640001ED00922C24C012905D0022908D10A2026
:1036500084F8E00114E084F8E021002068700FE0B5
:1036600084F8E021FFF7D0FE04EBD004A889FFF72F
:10367000CBFEB84900F00700085C217808432070B1
:10368000B149062048700120688130BD30B5AF4D8A
:10369000A889FFF7B9FEAE4901EBD004A889FFF76E
:1036A000B3FEAD4900F00700085C217808402070A7
:1036B000A549062048700120688130BD2DE9F04FF2
:1036C000DFF88492022189F8011099F8041099F822
:1036D0000300002701EB002080B2FFF758FEDFF85F
:1036E0006CA241F29071AAF80C0080B2884203D01B
:1036F000A0F5B852D03A60D188425ED197480024F4
:103700008046B0F800042646DFF854C2C5B223E074
:103710000CEB460000F58050B0F80404FFF737FECC
:103720000CEB440240083CF8101002F58052A2F85D
:103730009017641CA0F5C061A4B26E290AD80CEBE6
:1037400044010CEB4000408801F58051641CA1F855
:103750009007A4B2761CF6B2AE42D9D3B8F80204F0
:1037600000254FF0010B00F0FF0824E070190CEB6E
:10377000400000F58050B0F80404FFF745FE010951
:103780003CF8111000F00F020BFA02F28A4304EB2E
:1037900015110CEB410101F58051B1F8902705F0AE
:1037A0000F030BFA03F001D1024300E082436D1CCA
:1037B000A1F89027EDB24545D8D30020694CC84602
:1037C000DFF88CE1D446BAF80C509AF8056013E0A3
:1037D000291811F80E2004EB12110B7808EB4001A8
:1037E0008B7002F00F02A25CCA70C978DAB2114481
:1037F0003944401CCFB280B2B042E9D3032208EB77
:1038000040018A70FF1CFAB204EB12131B7802F01D
:103810000F02CB70A25C0A71042101EB4000ACF8EE
:103820000A00BDE8F08FF0B5474D484E2879E97899
:10383000002400EB0120B081454F09E0B08920440D
:1038400080B2FFF7A4FD29198979641CC155A4B27F
:1038500070798442F2D30620687001207081F0BD37
:103860002DE9F041DFF8E0C0022038498CF8010072
:10387000C8890022A0F5004086B2CE811046394D9D
:10388000DFF8E4E088464F7913E031181EF8013084
:1038900005EB13110C780CEB40018C7003F00F0357
:1038A000EB5CCB70C978E3B219441144401CCAB236
:1038B00080B2B842E9D303230CEB4001D21C8B70D9
:1038C000D2B205EB12131B7802F00F02CB70AA5C88
:1038D0000A71042101EB4000A8F80A0074E42DE904
:1038E000F047DFF86480194E98F8041098F8030048
:1038F000174F01EB002080B20A21B08187F8E01158
:103900004FF0010986F80190B0F5004F49D300212E
:10391000164AA0F500401170B0810C4606F1100562
:10392000134F3AE0B0890119C80A2870C2B268780A
:1039300082421FD108EB04005242807901EBC22180
:1039400027F8110027E000008C7E0020F400002002
:1039500000100020EC5F0008F45F00080020002049
:1039600000100020BA430108006000083B0000205E
:10397000886E0020FFF701FC2878FFF727FC2878E5
:103980006870B28908EB040122444042897902EB55
:10399000C02027F81010641CA4B270798442C1D3EF
:1039A00011E0001DB0810024454609E0B0892044A3
:1039B00080B2FFF7ECFC29198979641CC155A4B2C7
:1039C00070798442F2D3062188F80110A6F80A9093
:1039D000BDE8F08770B50522A0F50040F94B0C0A50
:1039E000CDB280B245F6DB66195CA94205D1191843
:1039F0004978A14201D1002201E0801C80B2B0428E
:103A000001D8032AF0D800F5004080B270BD70B52F
:103A1000ED4CEE4D6179A07901EB002081B2E8898F
:103A2000FFF7D8FFE881022060703120A070E8899C
:103A3000010AC2B2E64800EB11131B78E37001F0F3
:103A40000F01415C217100EB12110978617102F0E4
:103A50000F01415CA1710321E171D9B222793131A9
:103A6000114462791144A2791144C91CC9B200EB16
:103A700011121278227201F00F01405C607209206D
:103A8000688170BD30B50A280ED2D24BD24C0021CD
:103A90004FF4006501EBC02292B29A5C24F8112029
:103AA000491C89B2A942F5D330BD2DE9F05FC74E5C
:103AB00005468846B17000F500400F2180B2FFF73F
:103AC00089FF4044A0F5004084B25B2D2AD9A5F1BE
:103AD0005C0001044FEA115CB178A4F15C00490874
:103AE000C9B2C0F34E00C00801F00703CA08B370A2
:103AF000BA490BE00E1816F8016C0F5C06EB0726AE
:103B00009E40360A8718401ECE5580B26045F1D1DE
:103B10000E1816F8016C0F5C104406EB07269E4049
:103B2000330A0B544FEAD42AE00A8346B0EBD52F70
:103B300002D1C5F30A0700E00027BAEBD42F03D166
:103B4000C4F30A06761C01E04FF400665846FFF7FE
:103B50003DFB4FEAD42938464FEAC9299D4ADFF890
:103B600078C2731C0AE000BF09EB0001A1EB080159
:103B700089B2515C2CF81010401C80B29842F3D3EB
:103B80005846FFF7FAFAF01B201A84B205EB08003A
:103B9000A042C9D3BDE8F09F2DE9F0418A4F8B4E7A
:103BA0007879B979081A10F0FF0105D0F089A0F5ED
:103BB000004080B2FFF779FF89490020834D0870EB
:103BC0006420103528706870F97838794FF4004215
:103BD00002EB01210844B081B87900247071DFF84C
:103BE000F88121E0B0890119C80A2870C2B268784A
:103BF000824207D138195242C07901EBC22128F81C
:103C000011000FE0FFF7B9FA2878FFF7DFFA2878FC
:103C100068703919B28940422244C97902EBC02048
:103C200028F81010641CA4B270798442DAD3287882
:103C3000FFF7A3FA06207870012070814EE66349F1
:103C4000C8201031487008705F49062048705F49ED
:103C500001204881704710B55C4C10346078FFF744
:103C60008CFAC82060702070FCF7F3FE56490620DD
:103C7000487056490120488110BD70B5534B1889D2
:103C80000B281ED157490879372801D0382818D178
:103C90004F4A8C7914324D79145D555D04EB05144F
:103CA000CD79097A555D515C2D0305EB0121214445
:103CB0009981372802D1BDE87040BBE4BDE870406F
:103CC000E4E4FFF720FB40498878612830D010DC1D
:103CD000112824D007DCE0B101281DD010282FD1F5
:103CE000BDE870409FE541281FD0602828D1012001
:103CF00022E077281CD005DC62281CD063281FD165
:103D0000022019E087280DD0D12819D1BDE87040D4
:103D100042E7BDE87040D1E4BDE87040A0E5BDE8F1
:103D20007040DCE5BDE8704095E7BDE870406EE6A8
:103D3000BDE8704083E70320BDE87040FFF768BA34
:103D4000152048700120588170BD10B51F4806210C
:103D50001D4A048901235170438110BD70B5FFF7DE
:103D6000B2FA2048184DC078184C37283CD008DCEF
:103D700030281CD031281FD034280CD1FFF7E5FFA4
:103D800009E0382835D0422838D0452803D1687951
:103D90006071FFF772FF608922890121104302D10F
:103DA00015206870618100202081A17170BD287983
:103DB0006071FFF72CFCEEE728796071FFF7C8FB14
:103DC000E9E70000006000088C7E0020F40000207D
:103DD000BA43010800500008886E002000D200207D
:103DE0003B00002080800020FFF785FAFFF7CFFB23
:103DF000D1E7FFF780FAFFF7EAFBCCE7FFF72BFFED
:103E0000C9E71FB500900020ADF80400ADF806002A
:103E1000ADF80800ADF80C000C20ADF80A006946BA
:103E20009048FEF70BF91FBD10B501218CB0880337
:103E3000FDF7C4FA01210846FDF7B7FA8A4C20467F
:103E4000FCF790FC87488021001D01908748029074
:103E5000102003908F2004900020CDE905010790E9
:103E600008908901CDE909010B9001A92046FCF7D2
:103E7000EBFC012202212046FCF71BFD4FF496408B
:103E8000FFF7BFFF774C012240F225512046FEF795
:103E900056F9012280212046FEF769F901212046CA
:103EA000FEF743F96015ADF8000003208DF802001D
:103EB00018206F4C8DF8030069462046FDF73BF84B
:103EC0002015ADF8000004208DF803006946204657
:103ED000FDF731F80CB010BD63484438416841F437
:103EE00000514160416C4FF6FE72114041646149DE
:103EF0000120087070472DE9F0475A48001D0188DD
:103F0000DFF8749101F07F01C8B206270124594EF1
:103F100089F800104FF00008A9F5FA75052806D1B8
:103F2000A6F808806F707481FFF763F922E0022819
:103F300001D1348121E03089F8B9307901280CD1E0
:103F40004FF49640FFF75DFFA6F808806F7074810C
:103F5000FFF74FF986F804800CE000281DD14FF4DC
:103F60001650FFF74EFFA6F808806F707481FFF7B8
:103F700040F93471308900280FD030894F46401CF9
:103F800080B2308199F8001009F80010B0F5C87FB0
:103F900004D9A6F80A80A6F8088019E50328FCD9F8
:103FA000384410F8020C0328F7D13348FFF778F9AA
:103FB000F0703089314B391811F8012CF17803EB8E
:103FC000111C9CF800C0624508D101F00F01385C5B
:103FD000595C884202D1BDE8F047BFE61520687001
:103FE0007481BDE8F047FFF704B970B51D4C40F28D
:103FF000255529462046FEF759F9012805D12946BD
:104000002046FEF772F9FFF776FF08212046FEF7FB
:1040100043F9012806D108212046FEF744F920463D
:10402000FEF7DDF840F2277529462046FEF73EF9F7
:10403000012808D129462046FEF757F900222946D3
:104040002046FEF77CF840F2266529462046FEF71A
:104050002DF9012805D129462046BDE87040FEF71C
:1040600044B970BD00380140440002408D7E0020FC
:1040700000080140F400002080800020BA430108BD
:1040800070B5FF4DFF22134605F5807606E000BFB0
:1040900010F8014B54402A5D5A40335D491EF7D257
:1040A00043EA022070BD1FB500900020ADF8040067
:1040B000ADF80600ADF80800ADF80C000C20ADF826
:1040C0000A006946EF48FDF7B9FF1FBD38B5012169
:1040D0008804FDF77CF901210820FDF76FF94FF402
:1040E0000060ADF800000420E74C8DF8030069463D
:1040F0002046FCF720FF2015ADF8000003208DF8C6
:10410000020018208DF8030069462046FCF713FFD3
:104110004FF49640FFF7C7FFDA4C012240F22551D9
:104120002046FEF70CF801212046FDF7FEFFD74898
:104130000021A0F8041F0121A0F8F21E38BD2DE9CE
:10414000F04FDFF84C83DFF844E343469F78DE7896
:1041500098F8010006EB072259791C79DFF834A39F
:1041600089B041F26F7C0EEB4203A8F164094FF075
:10417000000B05287DD013DCC54C0128257801AC47
:104180003BD0022877D0032801D004286ED18DF8C7
:1041900004508DF8050048008DF806000020C3E0AB
:1041A000BB4EBA4FB578F678062806EB052507EB27
:1041B000450505F500557DD00F2857D0102855D15D
:1041C000B3496245C879097A03D884B201EB042463
:1041D0002C80B2F5FA5F07D32880A3F58053B3F89B
:1041E000600001EB002028808AF801B05E4654464A
:1041F0008AF806B000204D4623E18DF804508DF872
:1042000005008DF806708DF80760B3F8A000010A6C
:104210008DF808108DF80900062101A8FFF730FF7E
:10422000010ACAF808008DF80A108DF80B008AF808
:1042300001B055465E468AF806B000204F46235C22
:10424000A979401C4A1C7B54C0B2AA710728F6D930
:10425000012240F227718B48FDF771FF0020414693
:104260000E54401CC0B20A28FAD9EE7009B0BDE85D
:10427000F08FC0E0FFE78DF804508DF805008DF851
:1042800006708DF80760B3F88000010A8DF80810F9
:104290008DF80900062101A8FFF7F2FE010ACAF80D
:1042A00008008DF80A108DF80B0055465F468AF815
:1042B00001B000E071E08AF806B000204E46235CB1
:1042C000A979401C4A1C7354C0B2AA710728F6D9B8
:1042D000012240F227716B48FDF731FF0020414673
:1042E0000F54401CC0B20A28FAD9EF70BEE7131869
:1042F000634509D80EEB400505F500552E8804EB03
:104300004005370AEF702E71B3F5FA5F0AD30EEB52
:104310004303A3F58053B3F8605004EB40032E0A27
:10432000DE701D71401CC0B245468142DFD89DF849
:10433000061001A8C91CFFF7A3FECAF808009DF8E3
:104340000620010A0DF10703D1549DF8062002A9A9
:1043500050548AF801B08AF806B09DF806C0564657
:1043600000200CF1040C4F4606E0B179235C4A1C96
:104370007B54401CB271C0B28445F6D2012240F297
:1043800027714048FDF7DBFE002059462954401CA8
:10439000C0B20A28FAD9F17068E7624503D8A0B222
:1043A00001EB00202880B2F5FA5F03D3A0B201EB45
:1043B000002028808AF801B05E4654468AF806B08C
:1043C00000204D4618F80030A179401C4A1C6B545F
:1043D000C0B2A2710728F5D9012240F227712948FD
:1043E000FDF7ADFE5FF0000008F80060401CC0B2B1
:1043F0000A28F9D956E001EB0420A3F8A0008AF8B6
:1044000001B05E4654468AF806B000204FEA09051E
:1044100018F80030A179401C4A1C6B54C0B2A2713C
:104420000728F5D9012240F227711648FDF787FECB
:104430005FF0000008F80060401CC0B20A28F9D9FB
:1044400030E018F80030A179401C4A1C6B54C0B20F
:10445000A2710628F5D306210D48FFF711FEA060D2
:10446000A179020A6A54491CC9B26854491CA17155
:10447000012240F227710348FDF761FE00200BE0A6
:104480001B44010800480040000C014000100020BF
:10449000D88200200801002008F80060401CC0B24B
:1044A0000A28ECD9E670E1E62DE9F0415F4D287964
:1044B000002853D12878002601284CD15C4F2E705B
:1044C000B7F8040F002846D15A4CB7F8F21E2078EE
:1044D000884240D1A87808280AD909212046FFF748
:1044E000CFFDA860A27AC1B2914210D1617A09E0F1
:1044F00006215048FFF7C4FDA860E279C1B291429D
:1045000005D1A179B1EB102F01D1FFF718FEB7F853
:10451000040F01281FD12078B7F8F41E88421AD161
:1045200005214448FFF7ACFDA860A279C1B29142D1
:1045300011D16179B1EB102F0DD12079E1783E4A8C
:1045400000EB0120A2F89C0000202654401CC0B2C1
:104550000A28FAD9AE70AE7001202871BDE8F0814A
:104560002DE9F041354D40F2255631462846FDF7FC
:104570009DFE2E4C00B331462846FDF7B6FE20794D
:10458000D0B12846FDF72BFE61792A4FC0B2012633
:1045900009B93870667126493878B1F8F21E884238
:1045A0000AD12846FDF71BFEA1787854491CC8B2F1
:1045B000A070072800D3267008212846FDF76CFE5E
:1045C000012806D108212846FDF76DFE2846FDF793
:1045D00006FE40F2277631462846FDF767FE0128A1
:1045E00015D1144960786439095C401C6070284614
:1045F000FDF7F1FD6078A179884204D100223146AF
:104600002846FDF79CFD31462846FDF76EFE40F238
:10461000266421462846FDF749FE01289ED1214601
:104620002846BDE8F041FDF760BE97E7080100208D
:1046300000100020D88200200030002000480040F8
:1046400081070ED16421B0FBF1F201FB120131B9F7
:104650004FF4C871B0FBF1F201FB120008B9012060
:104660007047002070472DE9F05F05469846DDE968
:104670000AAB0023A0F5FC608C469146792802D352
:104680000120BDE8F09F4FF4FC64AB4EAB4F08E057
:104690002046FFF7D5FF08B1334400E03B44641CDB
:1046A000A4B2AC42F4D3ACF10100C6B20024A44FD2
:1046B000DFF890C20EE0385D40F2A321484303EBDF
:1046C000C0132846FFF7BCFF10B1012C00D1634492
:1046D000641CA4B2B442EED340F2A32109FB01F062
:1046E00003EBC0119748C8EB481240420144C2EBAB
:1046F000082001EB0011CAEB0A1001EB800000EB6F
:104700000B040120FCF700FDFCF7F3FE2046FCF74C
:10471000C3FEFCF7EEFE0020B3E770B54FF4C8759A
:10472000B0FBF5F303290DD2840706D14FF47A7458
:10473000B0FBF4F604FB160414B905FB13040CB922
:10474000521ED2B2024402EB90021A446423B0FB20
:10475000F3F0101A7C4A801E515C0844072190FB3C
:10476000F1F201FB1200C0B270BD2DE9FC47774A9F
:10477000774992F8E101CB79764E184212D006F6CD
:104780001A663088C3B27088C2B2CDE90023B088FF
:10479000C3B2F088C2B23089C1B27089FFF763FF3B
:1047A000BDE8FC8792F8E20189780842F8D0FCF76E
:1047B0006CFEDFF890810546B0FBF8F362481F46B7
:1047C000801E0188994239D003804FF4FC644FF475
:1047D000B77C4FF4B6790FE02046FFF731FF38B1D0
:1047E000634502D3A3F5B77304E0641CA4B205E0EB
:1047F000A3F26D13641CA4B24B45EDD8A6F8244E69
:104800000024DFF83CC111E0B6F8220EFFF718FFD4
:1048100028B1012C03D11D2B0AD31D3B04E01CF849
:104820000400984204D81B1A641CA4B21C2BEBD2BF
:10483000641CA6F8224E5B1CA6F8203E08FB17500D
:104840004FF46162B0FBF2F106F61A66B18002FB2A
:1048500011013C22B1FBF2F0708002FB101030809D
:10486000F088C2B23089C1B27089FFF756FFB081BB
:1048700096E710B501214FF0C050FCF7A8FD0120CC
:10488000FCF742FCFBF7A8FE0120FCF732FD4120BB
:10489000FCF7BBFC0028FAD04FF48070FCF73AFD1F
:1048A0000120FCF73CFDFCF72AFEFCF722FE01216B
:1048B0000846FCF7D3FDFCF71CFE47F6FF70FCF73B
:1048C000F7FDBDE81040FCF714BE10B50420FBF75F
:1048D000A9FE45F65A24A04206D0FFF7CAFF21469A
:1048E0000420FBF79BFE1AE001214FF0C050FCF7BB
:1048F0006EFD002041F28831401C80B28842FBD31B
:104900007B20FCF782FC10B97A20FCF77EFCFCF7D8
:1049100083FD01210846FCF7A1FDFCF7EAFD0E48E6
:104920000B4A41789278114341700C4A0178D27950
:104930001140017010BD00000085E2018033E101EB
:104940001B460108805101001601002000100020C4
:10495000EC5F000800100020E1110020F45F000867
:1049600010B586B001210420FCF728FD012148077D
:10497000FCF72DFD3020ADF8040000248DF8074031
:1049800001A92448FCF7D7FA3C20CDE90204022013
:10499000059002A90020FBF771FE02A91020FBF789
:1049A0006DFE01210020FBF781FE01211020FBF7A5
:1049B0007DFE01210020FBF791FE01211020FBF775
:1049C0008DFE00210846FBF7AFFE00210846FBF7ED
:1049D000AFFE01210020FBF781FE01211020FBF733
:1049E0007DFE06B010BD10B50B4C0020B4F8A01E23
:1049F000FBF79AFEB4F8A21E0020FBF799FE0121F6
:104A00000020FBF76BFE0121BDE810401020FBF7F2
:104A100065BE0000000801400010002030B591B0D4
:104A200001214FF40470FCF7C9FC01210846FCF792
:104A3000BCFC0F20ADF8000000248DF8034069464F
:104A40004848FCF778FA484D2846FBF78BFE474864
:104A500001904748CDE902044FF4C870CDE9040441
:104A60008020069040000790800008902020099048
:104A70000002CDE90A0401A92846FBF7E5FE012161
:104A80002846FBF70BFF01208DF834008DF8350028
:104A90004FF46020CDE90E040C94344C04208DF8C2
:104AA00040004C3C0CA92046FBF71CFC07230122CC
:104AB0000A212046FBF796FC072302220B21204601
:104AC000FBF790FC072303220C212046FBF78AFC0E
:104AD000072304220D212046FBF784FC01212046F8
:104AE000FBF732FC01212046FBF724FC2046FBF7B4
:104AF0003EFC2046FBF740FC0028FAD12046FBF79D
:104B000042FC2046FBF744FC0028FAD10121204654
:104B1000FBF745FC11B030BD10B5FFF77FFFBDE8D6
:104B20001040FFF71DBF70B50022114C114E114609
:104B30006425002004EBC00333F81130401CC0B2E0
:104B40001A446428F6D392FBF5F006EB410202F515
:104B50008042A2F81C0F491C0022C9B20429E8D3E4
:104B600070BD000000100140080002404C240140CC
:104B70003C8300200010002053EA020C00F0698002
:104B80002DE9F04B4FF00006002B1FBFB3FA83F561
:104B900003FA05F424FA05F65E4012BF1643B2FA92
:104BA00082F502FA05F4C5F120051EBF22FA05FCC4
:104BB00044EA0C04203556EA044C4FEA144418BF6A
:104BC000641C4FF000084FF00009904271EB030C99
:104BD00039D3002919BFB1FA81F701FA07F6B0FA03
:104BE00080F700FA07F6C7F120071EBF20FA07FC7E
:104BF00046EA0C062037B6FBF4FCA7EB0507103F8E
:104C000007F01F0BCBF120060CFA0BFB2CFA06F673
:104C100044BFB3460026202FA4BF5E464FF0000BD2
:104C20005BEA060C08BF4FF0010B19EB0B09ABFB5D
:104C3000027C48EB0608C01B06FB02CC0BFB03CC36
:104C400071EB0C01C1E70B46024641464846BDE800
:104C5000F08B13B54FF000004FF00001AFF3008070
:104C6000BDE81C407047B2F120030AD5C2F1200311
:104C700001FA02F120FA03F300FA02F041EA03011B
:104C8000704700FA03F14FF000007047B2F12003C3
:104C90000AD5C2F1200320FA02F001FA03F321FA47
:104CA00002F140EA0300704721FA03F04FF00001DF
:104CB000704770477047704710B500F009F80068FA
:104CC00010BD10B5044600F003F8046010BD0000EC
:104CD00001487047704700005C860020004870471C
:104CE0005C8600207546FFF7F9FFAE460500694671
:104CF000534620F00700854618B020B5FBF76CFA44
:104D0000BDE820404FF000064FF000074FF00008CC
:104D10004FF0000B21F00701AC46ACE8C009ACE84D
:104D2000C009ACE8C009ACE8C0098D46704704462C
:104D3000AFF300802046FBF73CFA000003494FF038
:104D40001800ABBE704700000900000026000200FA
:104D5000704700002DE9FF4D21F0004582B0174655
:104D60000C4634A6B5F1795F08DA2146029801F0C5
:104D700087F818B903CE06B0BDE8F08D029A234635
:104D8000214610460EF0BEF9824602462B48884660
:104D90000B460621784400F05BF8434652460EF07D
:104DA000B1F900908B463A462146059B02980EF0D9
:104DB000A9F907460C465B4641465046009A0EF05C
:104DC000A1F923463A460EF0EFFB8B4600904FF0D8
:104DD000FF32414650460FF0A8F9194A954205DACC
:104DE0005B46009A0EF0E0FB0CCE1DE0154A9542A2
:104DF00002DD15A230CA02E0A5F5001500242B46FD
:104E000022460EF0D1FB0746884603CE2B462246AB
:104E10000EF0CAFB04460D465B4641463846009AF2
:104E20000EF0C2FB2B46224606B0BDE8F04D01F065
:104E3000C5B80000000000000000F03F90F800003E
:104E40003333D33F0000E93F000000000000D23FB1
:104E50002DE9F041491E0D46044600EBC10103C98E
:104E600016461F4609E03B4632460EF04BF96D1ED2
:104E700004EBC5020CCA00F0BFFC35F00602F2D10B
:104E8000022D23D0042D11D0062D30D13B463246C1
:104E90000EF038F9D4E90A2300F0AEFC3B46324666
:104EA0000EF030F9D4E9082300F0A6FC3B46324668
:104EB0000EF028F9D4E9062300F09EFC3B4632466A
:104EC0000EF020F9D4E9042300F096FC3B4632466C
:104ED0000EF018F9D4E9022300F08EFC3B4632466E
:104EE0000EF010F90CCCBDE8F04100F085BCBDE837
:104EF000F08100002DE9FF4D82B003980E9F20F055
:104F00000040B0F1795F09DADDE9020100F0B8FF95
:104F100020B9DDE9020106B0BDE8F08DDDE902232C
:104F2000194610460EF0EEF883468A460B460246B6
:104F3000DDE902010EF0E6F880462648019153466D
:104F40005A4605217844FFF783FF04460D4622A602
:104F50009FB92B462246514658460EF0D3F80CCE48
:104F600000F04AFC4246019B0EF0CCF8DDE902233A
:104F700006B0BDE8F04D00F03FBC0CCE40460199B4
:104F80000EF0C0F806460F462B46224640460199D1
:104F90000EF0B8F804460D46DDE904014FF0FF328B
:104FA0000FF0C3F82B4622460EF0FEFA53465A463F
:104FB0000EF0A8F8DDE904230EF0F6FA3B4632467F
:104FC0000EF0F2FADDE9022306B0BDE8F04D00F084
:104FD000F5BF0000D0F70000495555555555C5BFE0
:104FE00002494FF000000FF06EB800000000F87F9B
:104FF00002494FF000000FF066B800000000F87F93
:10500000080000002DE9F04D14469FA2D2E90032BD
:1050100090B0C4E902320E929D4A21F00045019100
:10502000954204DC03C4002010B0BDE8F08D994A1D
:10503000994E7E44954229DAD6E90423974F0029F8
:1050400011DD0EF0B1FABD4202D0D6E9062305E02B
:10505000D6E908230EF0A8FAD6E90A230EF0A4FA3E
:1050600003C40120E0E700F0C7FBBD4202D0D6E94F
:10507000062305E0D6E9082300F0BEFBD6E90A23A3
:1050800000F0BAFB03C44FF0FF30CDE7844B9D42E4
:1050900077DC074683A00CC8294638460EF032F864
:1050A00082A20CCA00F0A8FB00F0EAFE029000F019
:1050B0006FFFCDE90401D6E904230EF023F82B4657
:1050C0003A4600F07BFFD6E9062307468846DDE92D
:1050D00004010EF017F82A0D012503920B46024633
:1050E000414638460EF060FAC4E90001032D37D07E
:1050F000C1F30A500399081A05EB45111139814291
:105100002EDA654806977844C43800EB0516D6E9D0
:105110000023DDE90401C3460DF0F4FF8A460B4687
:1051200002460890594606980EF03EFA0746884611
:105130000B460246594606980EF036FA5346089A30
:105140000EF032FAD6E9022383468A46DDE90401ED
:105150000DF0D8FF53465A460EF026FA6D1CBDE7F7
:10516000019800280BDA606880F0004060600E98BB
:1051700080F00040E0600298404255E701E002986C
:1051800052E7C1F30A52B2F58D6F0BD9A2F2694210
:105190003623B2FBF3F2474B7B4403EBC2030CCB49
:1051A0000DF0B0FF00F07C460D460B4632460EF087
:1051B000FBF941A7D7E9002380468A4629463046B5
:1051C0000DF0A0FFCDE90C013DA00CC829463046EA
:1051D0000DF098FF0A908B460CCF514640460DF0DB
:1051E00091FF074636A00CC80E46514640460DF0CA
:1051F00089FF80460D4633463A4659460A9800F0E4
:10520000FBFA06460F460B460246DDE90C0100F0AC
:10521000F3FADDE90C2383468A460EF0C5F93B46D6
:10522000324600F0CBFE2B46424600F0E5FA26A7B8
:10523000D7E9002305460E46514658460EF046F87B
:105240000CCF00F01DFC03220EF06FFF20A20CCA51
:1052500000F0D2FA00F014FE1FA7D7E900234FEAAE
:105260006008514658460EF031F833462A4600F0A1
:10527000C3FA0CCF0EF02AF819A20CCA00F000FCF9
:1052800003C44046D0E6000000000000000000001B
:10529000FB21E93F7CD90240A2F60000FB21F93F47
:1052A000FB21394183C8C96D305FE43F0000000035
:1052B0000000E03FBCF40000000000404544DB3F3C
:1052C00000000090B1BF1DBEA7A540A74A6A0540D7
:1052D0000000000000002240A7A540A74A6AE53F61
:1052E000E704243E4544DB3F2DE9FF4D06468AB0E6
:1052F0008C4821F00045DDF858B098460F460C4622
:1053000085421FDA2146304600F0BAFDD0B90BF1D4
:10531000010145EA0100304303D132462B4682A009
:105320000AE0BBF1010F04D1304621460EB0BDE8C2
:10533000F08D234632467EA003C80EB0BDE8F04D86
:1053400000F09EBB7C4885421FDB002F03DA84F00F
:10535000004488F0004879A00CC82146304600F08F
:105360002DFE04460E4677A003C843460C9A0EF065
:105370001BF902460B463146204600F03DFA064630
:105380000C4672A0D0E900180C9123463246214603
:1053900030460DF0B7FE0B460246CDE908010DF090
:1053A000B1FE024602906B488A460B4606217844BD
:1053B000FFF74EFDCDE906016648534606217844C5
:1053C0002030029AFFF744FDDDE908230DF09AFE34
:1053D000DDE9082382460591214630460DF092FE14
:1053E000CDE90001DDE905305246079900F004FAE5
:1053F000DDE900230DF086FE43460C9A00F0FCF92F
:10540000DDE908230DF07EFE43460C9A00F0F4F926
:10541000824651A00CC88846DDE900010DF072FEFD
:105420004346524600F0E8F9CDE906010B46024634
:105430002146304600F0E0F982463F4888468542E2
:10544000584634DB00F0A4FDCDE904010B460246CA
:105450004146504600F0D0F905468B464346524639
:10546000414650460DF04EFE5B462A4600F008FBD2
:10547000DDE906230EF098F82346324600F09EFD43
:1054800001220EF052FEDDE9042300F097FD0446F0
:10549000022000EAA7700D46C0F1010000F078FD7F
:1054A0002B4622460EB0BDE8F04D0DF02BBE012874
:1054B00002D15046414639E745464346002221463F
:1054C000304600F07BFDDDE9062300F077FD07465E
:1054D0008B4617A003C84346524600F0D1FA8046D7
:1054E00000220C462B4610460DF00CFE0EA20CCAF4
:1054F00000F082F906460D465B463A4621460020FA
:105500000DF000FE2B46324600F076F92346424667
:105510000DF0F8FD23460EB0BDE8F04D002200F07E
:105520006BB900000000303E000000000000F03FBA
:10553000000000000000F0BF2894E53F182D4454FF
:10554000FB21E93F075C143326A6813C00000000E4
:10555000000000008EF30000635555555555D53FAA
:1055600030B520A30CCB214D21F0004487B0AC42D4
:1055700003DCFFF7EFFB07B030BD1D4A944206D1B4
:1055800028B90120FFF79DFB1AA103C9F3E7944254
:1055900005DB07B0BDE8304001220EF0C6BD02AA0F
:1055A000FFF730FD10F003000AD001280BD00228CD
:1055B00010D102A80FC8FFF7CDFB81F00041DAE758
:1055C00002A80FC8D5E70123009302A80FC8FFF770
:1055D00091FCF2E70123009302A80FC8FFF78AFCB1
:1055E000C9E700000000000000000000FB21E93FC7
:1055F0000000F07F010000000000F87F30B521A31B
:1056000014CB224D21F0004387B0AB4203DC0023D2
:105610000093234627E01E4A934207D130B9012068
:10562000FFF74FFB1BA103C907B030BD934205DB59
:1056300007B0BDE8304001220EF077BD02AAFFF7A7
:10564000E1FC10F003000AD001280FD0022812D18B
:105650000123009302A80FC8FFF74CFC0FE00123C1
:10566000009302A80FC8FFF745FCDDE702A80FC8AA
:10567000FFF770FBD8E702A80FC8FFF76BFB81F0BC
:105680000041D1E70000000000000000FB21E93FDD
:105690000000F07F010000000000F87F70B50400FA
:1056A0000D4601D0012200E000220A430B4B22F0FC
:1056B00000429A1AD20F0AD109A20CCA0DF0EAFCD4
:1056C00005D20120FFF7FDFA07A103C970BD2946E5
:1056D0002046BDE870400DF0C5BE00000000F07F20
:1056E0000000000000000000010000000000F87F42
:1056F00030B516A314CB174D21F0004387B0AB4251
:1057000003DC0123009323461DE0134A934207D193
:1057100030B90120FFF7D5FA10A103C907B030BD99
:10572000934205DB07B0BDE8304001220EF0FDBC1E
:1057300002AAFFF767FC00F001000121A1EB400382
:10574000009302A80FC8FFF7CFFDE7E700000000B5
:1057500000000000FB21E93F0000F07F0100000095
:105760000000F87F01F0004321F0004181EA41028E
:1057700012F0FE4F08BF12F4600F00F02880A1F174
:105780006051B1F5801F1BDB02014FF0404C09D87E
:1057900003D208BF4FF0000C0AE000F000521CEBEF
:1057A000820C05D410F100504FF0804C41F1000103
:1057B000B1F17F6F06DA43EAC10343EA50707047E4
:1057C000184670474FF0FF0243EAC250704711F489
:1057D000801F01D118467047DFF818C041EA030165
:1057E00050EA01327FF404ACAFF3008021F4E00012
:1057F000704700008800000410B591EA030F48BF0D
:1058000083F000430DF1D886841A71EB030E05D2A4
:10581000121943EB0E03001B61EB0E01DFF880C190
:105820004FEA1154A4EB135E1CEA430F18BF9CEA25
:10583000445F7DD023EA0C0321EA045143F4801332
:10584000DEF1200C38D322FA0EFC10EB0C0023FA08
:105850000EFC41EB0C01CEF1200C03FA0CFC10EB1A
:105860000C0051F10001B1F5801FCEF1200C38D2AF
:1058700001EB0451BDE8104012FA0CF258BF70471A
:10588000401C38BF5FEA420218BF7047002814BFAF
:1058900020F0010041F100014FEA410313F5001F20
:1058A00038BF704728BFB1F1C0413E494FF00000FA
:1058B00048BF41F000417047012A43EB0302AEF1BB
:1058C000200EDEF11F0C32BF4FF0000C23FA0EF356
:1058D00010EB030041EB0451B4EB115FCAD0A1EB14
:1058E000045101F58011490801EB0451BDE8104055
:1058F0005FEA30000CD350F1000038BF12FA0CFC04
:1059000006D1C3E7401C38BF5FEA4202C4D1BDE7FD
:105910004FEA410313F5001F38BF704728BFB1F1AC
:10592000C04120494FF0000048BF41F0004170479E
:105930009CEA445F08D0BDE8104011EA5C0F04BF48
:1059400001F0004100207047012841EB0104012AC9
:1059500043EB030E644598BFE645DFF84CC0BDE855
:1059600010403FF63DABAFF30080012841EB010052
:10597000012A43EB0302904208D010F5001F04BF38
:105980000020704719464FF00000704791EA030F5E
:105990004FF0000058BF704704494FF000007047B7
:1059A0000000E0FF0000F07F110000040000F87F1D
:1059B0004FF0807212EB400F98BF12EB410F1DD8D1
:1059C000AFF3008050EA010204D488420DD6EFF311
:1059D000008070478142EFF3008020F0104038BF14
:1059E00040F0004080F3008870474FF0010238BF5C
:1059F000022A68BF002AEFF3008070471CF4502F82
:105A000000F0E8820EF0C1BB00B54FF4001E1EEBA3
:105A1000410F08BF002898BF1EEB430F08BF002AA4
:105A200026D85DF804EBAFF3008051EA030C06D4EE
:105A3000994208BF904210D6EFF3008070478B4226
:105A400008BF8242EFF3008020F0104038BF40F0E2
:105A5000004080F3008878BF70474FF0010C38BFDA
:105A6000BCF1020F68BFBCF1000FEFF3008070477C
:105A70005DF804EB1CF4502F3FF4B2AA0EF085BB86
:105A800070B5DFF8ECC33CEA111418BF3CEA1314FC
:105A900000F09B8081EA03050CEA111444EAD574F6
:105AA0001CEA131518BF11EA0C1F00F074804FEAAE
:105AB000C1214FEAC32341EA505143EA5253A4EBB8
:105AC000050404F17F7441F0004143F000434FEAC4
:105AD000C0204FEAC22200F0A9F846054FEAD020C4
:105AE00003EB244340EA41504FEAD12101EB03523A
:105AF00082EAC47116D05FEA460E38BF4FF04046C6
:105B000010D314BF00234FF0004350F1000041F1C7
:105B1000000110EAD37F4FF0804620EAD37018BF0F
:105B20004FF0404691EAC47FDFF848E316D412EA0A
:105B30000E0F18BF3EEA010E10D070BDE50754BF2E
:105B40001EF4000F1EF4800F0ABF4FF080464FF086
:105B5000404610F1010041F10001E3E7B4F1806F2C
:105B6000DEBF01F1C04101F00041002000DC70BD4A
:105B7000A8BFA1F1C04146F0140CA8BF4CF0805C56
:105B8000BDE870406FF0000041EA500181EA103139
:105B90004FF00000704711EA0C1F00D00AE013EA32
:105BA0000C1F00F03D804FF0000081EA030101F07E
:105BB000004170BD6FF0000081EA030141EA50012D
:105BC00081EA10314FF0000070BD4FEA410EBEEB8C
:105BD0004C1F4FEA430508BF002898BFB5EB4C1F88
:105BE00008BF002ABDE87040DFF88CC23FF6F8A974
:105BF000AFF300804FF4001C1CEB410F09D11CEBEC
:105C0000430F0FD04B4021F0004148BF41F000410D
:105C100070474FF0000081EA030303F00041704732
:105C2000BDE870404FF0000094497047E0B505466C
:105C300010B40C460FF238114FEA430C4FF0010E2E
:105C40004FEA9C6C51F82CC04FF00001ACFB026095
:105C50004FF00006ECFB0301001841EB0101301A84
:105C600066EB0101E1FB0C6C4FF00001ACFB026044
:105C70004FF00006ECFB0301001841EB0101301A64
:105C800066EB0101E1FB0C6C4FF00001ACFB056021
:105C9000ECFB0401A2FB0167E3FB006E17EB0E07B0
:105CA0004FF0000EE3FB017E4EF1000EB6197F416E
:105CB0004EEB0E0E764275EB070764EB0E0EECFB17
:105CC0000E01ACFB07E64FF0000E801941F1000118
:105CD000A2FB0067B619E2FB017EE3FB007E7F4179
:105CE00003FB01EE4EEB0E0E76424FF0000676EB14
:105CF000070765EB0E0EACFB0E674FF0000E4FEA88
:105D0000857C4FEA9505C01941F1000145EA84758B
:105D100049084FEA3000A2FB00677642E2FB017EB1
:105D2000E3FB007E7CEB070703FB01EE65EB0E0E49
:105D3000B51A77EB03047EF1000E24BF2E462746EA
:105D400050F1000041F10001012E38BF012F404108
:105D500041EB010111F0004F18BF022301D0F0BC4C
:105D600000BDF0BC4FF00103001841EB010100BD84
:105D7000FCC00FFC830F3EF85F8D89F4F0F0F0F06B
:105D8000B50373EDEAA00EEA48B4C2E6E3388EE349
:105D90001C3870E0A6C867DDA70D74DAE53594D726
:105DA000037BC7D4D2200DD2A87464CFCCCCCCCC8A
:105DB000E68745CA7C0CCEC77BC865C5C3300CC31B
:105DC000C0C0C0C00BFA82BE0B6452BCA28B2EBAFC
:105DD000E00217B8B6600BB6B4400BB4C84216B2B6
:105DE000020B2CB05C414CAE849176ACAAAAAAAA54
:105DF000573FE8A839052FA702B57EA53D0AD7A3CE
:105E00002BC337A2A0A0A0A0E765119F9DD8899DB4
:105E10009CC0099CD9E7909A511A1F99ED25B49717
:105E20006CDA4F964F09F294C4859A939224499262
:105E300009BCFD90EE23B88F6D35788E08CB3D8D73
:105E40008CC0088CFBF2D88A8940AE898888888803
:105E50005FAB67877D8A4B8653083485420821846F
:105E6000976E12838220088208040281000000805D
:105E70000000FF070000F07F140000040000F87F1E
:105E80004FEAC12303B40A1543EA505318BF43F045
:105E900000430DD4A2F56072D2F19E0240F321803E
:105EA000FF2ACCBF002123FA02F1084602B0704756
:105EB0004FEA4252520D08BF23F000434FF0000159
:105EC000A2F56072D2F19E020BDBFF2ADCBF23FA3F
:105ED00002FCA1EB0C010029DEBF02B008467047AE
:105EE000FFE703BCDFF830C0012841EB010313F5E5
:105EF000001F88BF4CF4803C3FF67AA83EBF6FEA93
:105F0000E17080F000407047AFF300806FEAE1700D
:105F100080F0004070470000C80002044FEAC1232F
:105F200003B40A1543EA505318BF43F000430CD49E
:105F3000A2F56072D2F19E0211DBFF2ACCBF0021D4
:105F400023FA02F1084602B0704701F1804212F5CF
:105F5000801F80F204804FF0000002B0704703BC45
:105F6000DFF828C0012841EB010313F5001F88BFAB
:105F70004CF4803C3FF63CA83CBF6FEAE1707047B0
:105F8000AFF300806FEAE17070470000E8000204A0
:105F900010F0004314BF4142014643F08043B1FA80
:105FA00081FC03F1F87311FA0CF1A3EB0C534FEAE7
:105FB000415008BF704703EBE121704791EA030F9E
:105FC00010B581F000413FF51FAC83F000430DF0A8
:105FD000F3BA000001480EF076B800000000C07F60
:105FE00001480EF070B800000000C07F01020408F4
:105FF00010204080FEFDFBF7EFDFBF7F00000000B8
:106000001000D8BA000000002020202020202020EE
:106010002020202020202020202020202020202080
:106020002020202020202020202020202020202070
:10603000F409FF0BF401E703640EC70EDC0EFF0E3C
:106040009001FE03000000000000000000000000BE
:106050008300000000000000000000000F00FFFFB0
:10606000FFFFFFFFFFFFFFFFFFFFFFFFFFFFFFFF40
:10607000FFFFFFFFFF000000000000000000000025
:106080000000000000000000000000000000000010
:106090000000000000000000000000000000000000
:1060A00000000000000000000000000000000000F0
:1060B00000000000000000000000000000000000E0
:10E4D00030B500230AE00D186D1E6D08AA4207D85A
:10E4E0001CB9091A491C03EB51032946012406E013
:10E4F0001CB1081A401C03EB5003681C002488421E
:10E50000E9D3184630BDF0B5002501231F4616E0BB
:10E510000C1A641C05EB54043E46A24200D30026AC
:10E520009E4206D003B125460844401C4008002303
:10E5300005E003B925460144491E490801238842E4
:10E54000E6D3F0BD0346012101E05B084900002B42
:10E55000FBD109B9581E7047491E02460020B7E793
:10E560000346012101E05B084900002BFBD109B9FA
:10E57000581E7047491E02460020C4E770B5FB4C88
:10E58000FB4DA06D2844C0F34F0003F087FF002827
:10E590006079F84A4FEAC07013D128B3A06D4119D1
:10E5A0004810C31700EB537002EBE00220F00700A5
:10E5B000C0EB6100F0491378405C03431370012005
:10E5C00070BD88B9A06D41194810C31700EB537096
:10E5D00002EBE00220F00700C0EB6100E64913788F
:10E5E0000831405C03401370002070BDE3480022F6
:10E5F000A0F8182EB0F8882E4AB9A0F8861EDB497C
:10E60000DB4AC96D521E11444910A0F8881EB0F8AB
:10E61000881EA0F88A1E704770B5D94BD34A03EB09
:10E62000D00100F0070610464079D34C4006097827
:10E63000A65D157B000E3140012D50710ED10029D1
:10E640000BD0118C03EBD10301F007011B78615C47
:10E650000B4202D040F00100507170BD0029F9D189
:10E6600070BD70B5C64BC14A03EBD00100F0070680
:10E6700010464079C04C40060978A65D157B000E17
:10E680003140012D50710FD100290CD1118C03EBB9
:10E69000D10301F007011B78615C0B4203D000BF7E
:10E6A00040F00100507170BD0029F9D070BDB4492F
:10E6B00001EBD0010A78B04900F00700085CAB49D3
:10E6C0000242487904D0C20702D040F0010001E0C4
:10E6D00000F0FE0048717047A94901EBD0010A78AB
:10E6E000A54900F00700085CA0490242487904D11E
:10E6F000C20702D040F0010001E000F0FE004871C6
:10E7000070479F4901EBD0010A789B4900F0070050
:10E71000085C96490240487900F001031A4302D090
:10E7200040F0010001E000F0FE004871704794499C
:10E7300001EBD0010B78904900F00700085C8B4991
:10E740000340487900F00102521E134202D140F00A
:10E75000010001E000F0FE0048717047F0B5DFF8FD
:10E760000CC2854F61464B799CF80D4084490837AF
:10E77000814D00F0070201EBD001012C2DD19CF856
:10E780000C40012C24D16446268C7D4C0A2804EBD5
:10E79000D60406F0070606D2D80716D02078BB5D4F
:10E7A000184020701BE02478AE5D34420DD0DB07AA
:10E7B00019D00B78AA5C13430B709CF80E10714AA9
:10E7C0004B1C22F811008CF80E30F0BD0870F0BD23
:10E7D0000A2802D2D807FAD001E0D80703D0087877
:10E7E000AA5C1043F2E70878BA5C1040EEE72DE926
:10E7F000F0435E4A5179C90732D0137BDFF880C1FC
:10E80000DFF8749100F007060CEBD001012B29D141
:10E81000002009F10805DFF86CE19046977B0BE0DA
:10E820003EF810400CEBD40204F0070413782C5D82
:10E830002340401C1370C0B2B842F1D9B8F8200090
:10E840000CEBD00200F007001478285C0440147030
:10E85000087819F8062010430870002088F80E0088
:10E86000BDE8F083087819F8062010430870F7E730
:10E8700010B53E4901224A730A7308844879404B17
:10E880004006020E4A71088C3B4C03EBD00300F0AB
:10E8900007001B78205C034202D042F0010048715F
:10E8A00010BD30B4314AF8385179947901F0FE0343
:10E8B00004F001051D43082820D2DFE800F0040918
:10E8C0001014161A1F0E41F0FE0000EA510003E07A
:10E8D00001F0010040EA5100507130BC704764F310
:10E8E0005F019171F9E75571F7E755716008907113
:10E8F000F3E70120884303435371EEE730BC022164
:10E900004FF4746072E62DE9F041184C1A4E6079AC
:10E910002146174F896D174DC00706F1080601EB18
:10E9200007003ED0C0F34F0003F0B8FD1449E0B932
:10E93000A26DD3195810C61700EB567005EBE00511
:10E9400020F00700C0EB63030B482E781B5C1E43CE
:10E950002E70128822F4504301EBD30102F007021B
:10E960000B78805C03430B7029E00DE03000002041
:10E97000A49FFFF7CD070020EC5F000800100020E7
:10E9800000100020AC050020A06D008820F450424B
:10E9900001EBD20100F007000A78305C02400A70F7
:10E9A0000DE04110CA1701EB527105EBE10221F0B5
:10E9B0000701C1EB60001378805D03401370A06D08
:10E9C000801CA065BDE8F0812DE9F041F84CFB4EBC
:10E9D00060792146896DC007F64DDFF8DC8301EBD5
:10E9E0000600C0F34F0013D003F058FD90BBA06D9C
:10E9F00081194810C21700EB527005EBE00220F0BD
:10EA00000700C0EB6100137810F8080003432DE005
:10EA100003F044FDE849EA4A0831E0B1A36D1E4421
:10EA20007010C71700EB577005EBE00520F00700EA
:10EA3000C0EB66002F78405C07402F70188820F4E8
:10EA4000504102EBD10100F007030A7818F80300E7
:10EA500002430A700BE0A06D008820F4504302EBE3
:10EA6000D30200F007001378085C03401370A06D18
:10EA7000801CA065A6E72DE9F041DFF834E3A0F1A2
:10EA8000820CDEF8603043EA0222BEF810301A44ED
:10EA900002F01F04CEF8602052099204160C0023E5
:10EAA000BCF10F0F51D2DFE80CF0085010501A5093
:10EAB00023502B5033503C50450001F00F001946B5
:10EAC0002246F6F7D0F80F2205E0C8B219462246D2
:10EAD000F6F7C9F8FF22A240D743FD173AE0C1F389
:10EAE0000B0019462246F6F7BEF840F6FF72F2E731
:10EAF00088B219462246F6F7B6F84FF6FF72EAE7F3
:10EB0000C1F3130019462246F6F7ADF8AD4AE2E725
:10EB100021F07F4019462246F6F7A5F86FF07F42B4
:10EB2000D9E721F0704019462246F6F79CF86FF0BD
:10EB30007042D0E708461D4622461946F6F793F87C
:10EB40004FF0FF32A240D74304E0DEF85820921D78
:10EB5000CEF858209A4A3244D2E900343B402C4047
:10EB600003430C4318C22DE710B591490A6E01F119
:10EB7000800442EA00200A8A104400F01F0208665E
:10EB8000400980044A82000C88828D49014403C9EF
:10EB9000F6F77CF803C410BD10B5854B996D8A1C3F
:10EBA00009880C0A803C092C15D2DFE804F0051412
:10EBB0000B1416141C14220000EB012080B24FF439
:10EBC000E06104E000EB012080B24FF4006101EB52
:10EBD0005000D8829A65D88A10BD00EB012080B21F
:10EBE0004FF4A061F3E700EB012080B24FF48051B5
:10EBF000EDE700EB012080B241F2E831E7E710B524
:10EC00006B4CA06D811C0088020A842A09D0862AD8
:10EC100005D1C0B26070A165FFF7BEFF2083208BD5
:10EC200010BDC0B2607031F8022B40EA0220208390
:10EC30000020A1652070F2E770B55D4CA06D821CCC
:10EC40000388A265418803F47F40DBB20D0623668A
:10EC500040EA112043EA1543A0F50645803D01D165
:10EC6000594818E0A0F50645823D03D103F1202361
:10EC7000A36212E0A0F50645843D01D153480AE0A5
:10EC8000A0F50645863D01D1514804E0A0F50645B2
:10EC9000883D05D14F481844A062921CA26550E0FF
:10ECA0000025A0F50442823A05D1C8B2FFF75CFF07
:10ECB00000F00F0040E0A0F50442843A04D1C8B24D
:10ECC000FFF752FFC0B237E0A0F50442863A05D103
:10ECD000C8B2FFF749FFC0F30B002DE0A0F50442D6
:10ECE000883A04D1C8B2FFF73FFF80B224E0A0F514
:10ECF00004428A3A05D1C8B2FFF736FFC0F31300C9
:10ED00001AE0A0F504428C3A05D1C8B2FFF72CFFF7
:10ED100020F07F4010E0A0F504428E3A05D1C8B241
:10ED2000FFF722FF20F0704006E0A0F50442903A81
:10ED300007D1C8B2FFF718FFA0622570A06D801C34
:10ED4000A065A06A70BD2449800B02D1B1F83A0ECB
:10ED50007047012802D1B1F86E0F7047022802D126
:10ED6000B1F8720F7047032802D1B1F8760F7047DF
:10ED7000002070471849800B02D1B1F87A0F704714
:10ED8000012802D1B1F87E0F7047022802D1B1F8F4
:10ED9000820F7047032802D1B1F8860F7047002018
:10EDA00070470D49800B19D1B1F8380E704700003B
:10EDB00030000020CD070020EC5F0008A49FFFF783
:10EDC00000100020FFFF0F00001E0020001A00208E
:10EDD00000300020D037002000100020012802D190
:10EDE000B1F86C0FE2E7022802D1B1F8700FDDE74D
:10EDF000032802D1B1F8740FD8E70020D6E7F8490C
:10EE0000800B02D1B1F8780FD0E7012802D1B1F818
:10EE10007C0FCBE7022802D1B1F8800FC6E70328A8
:10EE200002D1B1F8840FC1E70020BFE7EC49800BA5
:10EE300004D1B1F8380EB1F83A1E13E0012804D11C
:10EE4000B1F86C0FB1F86E1F0CE0022804D1B1F8D4
:10EE5000700F00EB0040A9E7032806D1B1F8740F4A
:10EE6000B1F8721F00EB0140A0E700209EE7DC4AEA
:10EE7000800B04D1B2F8780FB2F87A1F12E00128A3
:10EE800004D1B2F87C0FB2F87E1F0BE0D4490228FF
:10EE9000B1F8821F02D1B2F8800F03E0032805D138
:10EEA000B2F8840F00EB014080B27FE700207DE7DD
:10EEB0002DE9F047CB4DDFF83093A86DDFF82C83B8
:10EEC00000F1020C0088C5F858C0BCF8007000F4CE
:10EED0007F4141EA1724C3B239062B6643EA114346
:10EEE0004AF28741601A8C426FD045DCBD4E48F231
:10EEF0008262716E368AA4EB0200944266D024DCF2
:10EF000048F28A42A4EB02004FF00108944259D023
:10EF10000CDCA4F50444823C44D0022C45D0042CE3
:10EF20004DD0062C76D1FAB2882040E0022849D094
:10EF3000042847D0062845D0B0F5FB7F6AD19A193E
:10EF400002EB0900C0F8001E44E041F60167C21B55
:10EF5000B84268D009DC022841D0042845D00628F0
:10EF600048D0B0F5F05F55D159E0012A57D0022AB8
:10EF700059D0032A4ED152E00A2854D008DC0A287E
:10EF800048D2DFE800F0474C504C504C504C504CAD
:10EF9000A0F2FB1008283DD2DFE800F0494D575B96
:10EFA000696D7A7EFAB2822001E0FAB28420FFF71E
:10EFB00062FDA86D801CA86585F809802AE0FAB278
:10EFC0008620F4E7FAB2E0B2F1E72CE0981900F1FC
:10EFD00020200DE00CF1020CC5F858C01AE09A1977
:10EFE00002EB0900C0F8001AF4E79A1902EB0800D6
:10EFF0000160EFE79A1902EB0800C0F8D017E9E7C3
:10F000002866C3F30522E0B2696EFFF734FDA86DF0
:10F01000801CA865A86D001DA865BDE8F08718468E
:10F02000FFF704FFECE71846FFF721FFE8E7184673
:10F03000FFF7FCFE02E01846FFF719FFC3F30D01CE
:10F0400001EB400000F120201EE01846FFF7EEFE25
:10F0500002E01846FFF70BFFC3F30D0101EB40017F
:10F0600001EB0900696E89B2C0F8001ACFE71846B3
:10F07000FFF7DCFE02E01846FFF7F9FEC3F30D01CF
:10F0800001EB400101EB0800696E89B20160BEE747
:10F090001846FFF7CBFE02E01846FFF7E8FEC3F381
:10F0A0000D0101EB400101EB0800696E89B2C0F867
:10F0B000D017ACE72DE9F0474A4CDFF82C91A06D52
:10F0C000DFF8288100F1020C0088C4F858C0BCF8B1
:10F0D00000E000F47F4141EA1E23C2B24FEA0E6114
:10F0E000226642EA114249F28561581A4FF4FD7ACC
:10F0F0008B4274D053DC49F28341A3EB01008B4275
:10F100003ED032DC374848F28266416E008A89B2CE
:10F11000A3EB06050FB2B3426AD01CDC48F2864668
:10F12000A3EB06054FF00108B3427ED009DCA3F53E
:10F130000443823B7AD0022B79D10EF0FF02842067
:10F1400091E0022D71D0554571D1111801EB0900E4
:10F15000A0F8007EA5E0022D6AD0042D69D0062D0E
:10F1600068D0B5F5606F62D1ADE00528FCD008DC51
:10F1700001286FD00228C3D003286BD0042856D1B1
:10F18000A5E0062867D0A0F58070FF3873D001286D
:10F1900072D002284BD11046FFF7D5FDABE040F608
:10F1A0000365A0F60361A84218D02BDC40F6FE559B
:10F1B000A0F6FE51A84224D01BDC032876D007DC41
:10F1C000012874D0022832D11046FFF7D3FDD9E0D0
:10F1D00004286DD0A0F55060FD3828D1B1E087E05B
:10F1E000001000203000002000100020003000201F
:10F1F00043E00129F2D00229DDD003296FD0042990
:10F2000015D1A2E040F2FD15A1F2FD10A94267D090
:10F2100014DC012978D0514577D0A1F58071FB39F4
:10F2200074D0012903D1104605E019E014E021E073
:10F2300027E02CE030E0FFF7B4FD5CE001287DD052
:10F2400002287CD003287BD0042813D11046FFF776
:10F25000D6FD67E037E03AE00EF0FF02822002E0E0
:10F260000EF0FF02D8B2FFF706FCA06D801CA0656F
:10F2700084F80980D1E62EE033E0104400F120202C
:10F2800008E0111801EB0900A0F8007A09E0111854
:10F2900001EB0800078004E0111801EB0800A0F85A
:10F2A000D0770CF1020CC4F858C0B6E633E02EE07B
:10F2B00035E000BF2066606EC2F3052281B2D8B28D
:10F2C000FFF7D9FB36E01046FFF73DFDF2E71046A9
:10F2D000FFF750FDEEE71046FFF735FD40E030E068
:10F2E00045E01046FFF746FD3AE0606E088021E0F9
:10F2F0001046FFF73FFDC2F30D0101EB4001494409
:10F30000606EA1F8000A15E01FE022E025E010463B
:10F31000FFF719FD36E01046FFF715FD02E0104635
:10F32000FFF728FDC2F30D0101EB40014144606E7F
:10F33000A1F8D007A06D801CA0656EE61BE01EE062
:10F3400026E01046FFF72DFDB4E71046FFF757FD06
:10F35000B0E71046FFF725FD02E01046FFF74FFD2E
:10F36000C2F30D0101EB400101F12021BDE7104680
:10F37000FFF745FDBFE71046FFF713FD02E010461B
:10F38000FFF73DFDC2F30D0101EB40014144ACE745
:10F390001046FFF706FDC5E72DE9F04FF94C85B0A3
:10F3A000A16DDFF8E4A30B88881CA0654A8803F4EC
:10F3B0007F41914641EA12211206150CDAB222660B
:10F3C0002A4349F284654B1BDFF8C083A9427ED0F3
:10F3D0007EDCDFF8BCE349F28705BEF83A6EBEF882
:10F3E0006E7F0496BEF8726F0397BEF876BF0296E2
:10F3F000BEF87A6FBEF87E7FBEF882CFBEF886EF89
:10F40000A1EB0503A94275D04EDCDE4B48F2866EB7
:10F410001B8AA1EB0E0571456DD02EDC48F28647A4
:10F42000A1EB07064FF00105B9427DD014DCA1F530
:10F430000041803979D0B1F5007FFBD0A1F5806122
:10F44000023973D0022972D109F0FF00FFF78CFB5B
:10F45000C0B26083A572C1E1022E69D0B6F5FD7F0E
:10F4600067D0B6F5FE7FD7D0B6F5FF7FEBD11A4453
:10F4700002EB0A01B1F8001AB3E140F6FD1EA5F651
:10F48000FD11754528D00ADC022D7ED0A5F510654A
:10F49000FA3D7BD0012D7AD0022DD4D135E101295E
:10F4A00076D0022975D0B7E0B3F57F7F72D023DC28
:10F4B00040F2FD15A3F2FD11AB42F1D00DDCA3F536
:10F4C0008073F93BE5D0012BE5D0022B01E055E13B
:10F4D00042E0E3D0032BB6D18BE10129E2D002292F
:10F4E00070D003298FD0B1F5FF7FACD11046FFF764
:10F4F0002AFC12E101E1F0E040F20141A3F20140F7
:10F500008B427ED01BDCA3F54073FD3B7AD0012BF0
:10F5100079D0022B78D0032B95D11046FFF72AFC27
:10F520002066C2F3052005E0C2E0ADE0B2E07AE07B
:10F53000C7E0CBE0FFF718FBC0F30B004DE101285B
:10F540006FD0B0F5FD7F6DD0A0F58070FB386AD12B
:10F550001046FFF70FFC6DE1DFF834C240F60145BD
:10F56000BCF87C6FBCF8807F0196BCF884BFA3F622
:10F5700001410097AB4270D056DC8549B1F8389E06
:10F58000B1F86C5FB1F8706F05E0AAE0B9E0BAE0DD
:10F5900096E0B0E0BEE0B1F874EFB1F878CFB3F523
:10F5A000206F3BD01ADC052B70D00CDC012B6ED009
:10F5B000022B6DD0032B6CD0042B74D11046FFF7B7
:10F5C000C2FB02E12AE0A3F51063FC3B1ED0012B35
:10F5D00075D0022B74D0032B65D18FE040F6FD3738
:10F5E000A3F6FD31BB42F3D012DCA3F52063013B4F
:10F5F000C1D0012B6FD0022B6ED0A3F58073FB3BE3
:10F6000003E0A8E091E098E0A1E04CD149466EE02B
:10F6100001296ED0022971D0032944D10CEB0201DB
:10F62000DFE09CE0A4E03EE0B1F5017F6FD021DC9B
:10F6300040F2FF15A1F2FF13A94269D00EDC0129A7
:10F6400067D00229D8D0A1F58071FD3971D0012988
:10F6500029D11046FFF7D3FB5FE0C6E0012B69D04C
:10F66000022B68D0032B67D0042B1CD11046FFF768
:10F6700098FB77E0A1F2FD31082914D2DFE801F010
:10F68000D3D7E1E5F3F7F0EF62830AE09AE081E097
:10F690008BE093E009F0FF00FFF766FA00F00F003F
:10F6A000D7E6801CA065B4F91A0005B0BDE8F08F5C
:10F6B00009F0FF00FFF758FAC0F30B00C9E68FE02E
:10F6C00017E009F0FF00FFF74FFAC2E6D1185144E6
:10F6D000B1F8001E85E086E08BE01A4432F808108D
:10F6E0007FE01A4402EB0801B1F8D01779E0114429
:10F6F00077E0B11875E0B91873E0FFE70EEB02018F
:10F700006FE00499F3E70399F1E70299EFE786E0E8
:10F7100075E06CE01046FFF72DFB2066C2F3052074
:10F72000FFF722FA00F00F0057E01046FFF70BFB3F
:10F7300006E060E067E06AE06DE01046FFF71AFB64
:10F740002066C2F30520FFF70FFAC0B245E010466D
:10F75000FFF7F9FAE4E61046FFF7F5FA02E0104683
:10F76000FFF708FB2066C2F30520FFF7FDF934E040
:10F770001046FFF7E8FA5DE000882EE01046FFF73C
:10F78000E2FA0AE0300000200010002000300020E3
:10F79000001000201046FFF7EDFAC2F30D0101EB57
:10F7A00040005044B0F8000A17E01046FFF7CBFACB
:10F7B000C2F30D0101EB40004044DDE71046FFF7C6
:10F7C000D9FA57E01046FFF7D5FAC2F30D0101EB65
:10F7D000400101EB0800B0F8D0076083A06D60E73E
:10F7E000A91861835DE7009981E701997FE73946B0
:10F7F0007DE759467BE71046FFF7D3FA8DE71046C1
:10F80000FFF7CFFA9CE71046FFF7F9FA98E71046A2
:10F81000FFF7C7FA84E61046FFF7F1FA80E61046D4
:10F82000FFF7EDFA9EE71046FFF7BBFA02E010463D
:10F83000FFF7E5FAC2F30D0101EB400000F12020D3
:10F840009AE71046FFF7ADFA02E01046FFF7D7FA45
:10F85000C2F30D0101EB400101EB0A00A2E714E045
:10F860000FE004E0FFE71046FFF79BFA02E01046C6
:10F87000FFF7C5FAC2F30D0101EB400101EB0800EF
:10F880007AE71046FFF78DFA9FE71046FFF7B7FAC1
:10F890009BE72DE9FE4FFA4DDFF8EC93A96D4AF294
:10F8A0008426881C0B88A865804603F47F404A881C
:10F8B000DBB22B66B9F8784FB9F87C7F029440EA46
:10F8C0001221B9F8804F1006019743EA1043B9F8A6
:10F8D00084BF881BDFF8ACA3009405F16C04B1422F
:10F8E0006FD07ADC48F28666A1EB0600B14275D093
:10F8F00044DC48F28A47A1EB07004FF00106B94209
:10F900006DD020DC48F28447A1EB0700B94267D0F4
:10F9100010DCA1F5004180397BD0B1F5007FFBD030
:10F92000A1F58061023975D1D0B2FFF71DF900F061
:10F930000F0015E002286ED00428F4D1D0B2FFF7F2
:10F9400013F980B20CE0B0F5FB7F76D00BDC022817
:10F9500074D0042873D00628E5D1D0B2FFF704F99B
:10F960002060AE72F7E1B0F5FC7F69D0B0F5FD7FA5
:10F97000D9D1C6481844D0F8000A0BE1C24E41F66E
:10F98000FF17B6F838EEB6F86CCFB6F8702FC11B7B
:10F99000B6F8746FB8427AD023DC41F6FC17A0EBBE
:10F9A0000701B84274D008DC022872D0A0F5C85014
:10F9B000FA3822D00128B6D1F7E0012932D0022945
:10F9C000B1D102984E461844208008F10200A86583
:10F9D000FFF7E2FCB6F87A1F54E032E0DDE0BDE06C
:10F9E000B1E0B1F5FE7FE7D016DC01297ED0022917
:10F9F0003DD0A1F58071FB3995D10EEB030020803D
:10FA000008F102004E46A865FFF7C6FCB6F83A1E9C
:10FA100038E08EE0B5E09BE0A1F58071FD39C1D002
:10FA200001298AD1F018208008F102004F46A8650C
:10FA3000FFF7B2FCB7F8761F24E0A3E094E099E06A
:10FA4000A5E04FF4FF77B0F5027F79D034DC40F2C7
:10FA50000122A0F20121904273D025DCB84271D07E
:10FA600018DC012897D00228C0D00328A3D10BEBC3
:10FA70000300208008F102004E46A865FFF78CFCC9
:10FA8000B6F8861F08446080A86D001F65E1A7E0F6
:10FA90009BE085E0A0F58070FF3871D001288AD105
:10FAA0001846FFF7C3F9C7E007296AD2DFE801F07B
:10FAB00069CBCFDADEF2F60040F2FF320026A0F288
:10FAC000FF3141F6322940F6437B904279D024DC65
:10FAD000B0F5037F76D014DCA0F50070093872D041
:10FAE000012871D0022887D1184600E085E0FFF791
:10FAF000BEF92866C3F30520FFF736F820F0704002
:10FB000095E0A0F500700D3876D0A0F58070F13842
:10FB100087D11846FFF78AF9F2E043F67E6C43F28C
:10FB2000AE680729C1D2DFE801F02CF9F7F6F5F449
:10FB3000F300238008F10200A865FFF72DFCA2E77F
:10FB4000B7E076E065E0D0B2FFF70EF8C0B207E7A5
:10FB5000D0B2FFF709F8C0F30B0001E7D0B2FFF70E
:10FB600003F8C0F31300FBE6D0B2FEF7FDFF20F070
:10FB70007F40F5E6D0B2FEF7F7FF20F07040EFE6E9
:10FB80004BE0EBE041481844D0F8000E02E003F1EE
:10FB90002023186820604046DEE053F80A00F9E7A9
:10FBA00003EB0A00D0F8D007F4E70CEB0300208049
:10FBB00008F102004E46A865FFF7EEFBB6F86E1F8F
:10FBC00060E79AE088E078E082E0D018208008F1D1
:10FBD00002004E46A865FFF7DFFBB6F8721F51E73B
:10FBE00001984E461844208008F10200A865FFF7EE
:10FBF000D3FBB6F87E1F45E772E000984E461844E6
:10FC0000208008F10200A865FFF7C6FBB6F8821F46
:10FC100038E71846FFF70AF902E01846FFF727F918
:10FC20002866C3F30520FEF79FFF00F00F00206059
:10FC300091E01846FFF71BF92866C3F30520FEF78D
:10FC400093FFC0B2F3E71846FFF7F0F802E018465A
:10FC5000FFF70DF92866C3F30520FEF785FFC0F313
:10FC60000B00E4E71846FFF7E1F802E01846FFF75B
:10FC7000FEF82866C3F30520FEF776FF80B2D6E7CC
:10FC80003000002000300020001000200010002074
:10FC900004E0FFE71846FFF7C9F802E01846FFF74F
:10FCA000E6F82866C3F30520FEF75EFFC0F31300F5
:10FCB000BDE71846FFF7BAF802E01846FFF7D7F895
:10FCC0002866C3F30520FEF74FFF20F07F40AEE724
:10FCD0001846FFF7ABF80CE71846FFF7A7F802E065
:10FCE0001846FFF7C4F82866C3F30520FEF73CFF6B
:10FCF0009DE700BF00F1202037E01846FFF7B7F876
:10FD0000C3F30D0101EB400080B2B842F2D347E0EB
:10FD10003CE037E02BE015E009E0FFE71846FFF78D
:10FD200085F807E0FF490844D0F8000A7FE7184645
:10FD3000FFF79DF8C3F30D0101EB400080B2B8421C
:10FD4000F0D32DE01846FFF771F813E04946584606
:10FD5000FEF74CFC2660A86D801CA865A86D001DF0
:10FD6000A8652068BDE8FE8F504400685FE718462C
:10FD7000FFF77DF8C3F30D0101EB400080B2604551
:10FD8000F2D3E3E71846FFF751F802E01846FFF711
:10FD90006EF8C3F30D0101EB400080B2404505D37E
:10FDA00049465846FEF722FC2660D7E75044D0F873
:10FDB000D0073CE72DE9F041DB4DA86D05F16C075C
:10FDC000838841880288841DAC65C68802F47F4020
:10FDD00040EA11200906D2B242EA11413206DBB2F2
:10FDE00043EA12423E1FA0F50043803B02D0B3F528
:10FDF000007305D139807A80386803F065FF26E00A
:10FE0000C84AA0F50643803B03D18818D0F8000EFD
:10FE10001DE0A0F50643823B03D101F120210868D3
:10FE200015E0A0F50643843B03D18818D0F8000AFA
:10FE30000DE0BE4AA0F50643863B01D1885806E096
:10FE4000A0F50643883B05D18818D0F8D007A41C3C
:10FE50003060AC653068BDE8F0812DE9F047B2490B
:10FE60004879C0074DD0FEF7CAFE8046FEF7C7FEB0
:10FE70008246FEF7C4FE8146FFF78EFA1FFA80FE27
:10FE80000021DFF8ACC2A74F37E000BF0AEB010446
:10FE900007EBD40004F0070403781CF80440C1EB1E
:10FEA000C10223430370002002EB090208EB0004A7
:10FEB00007EBD40304F007041B781CF8044023422A
:10FEC0000AD0131807EBD30403F0070325781CF8B6
:10FED00003301D4325700AE0151807EBD503944E37
:10FEE00005F0070508361C78755D2C401C70401C19
:10FEF000C0B20728DAD9491CC9B27145C6D3BDE8DA
:10FF0000F087886D10308865F9E770B5864D68799F
:10FF1000C0072CD0FFF740FA6866FFF7CBF8FFF771
:10FF20003BFA0646A86D001F0124A86517E0A87AD1
:10FF3000012801D1200100E060002882A86D083866
:10FF4000A865FFF729FA6866687A012801D12001BF
:10FF500000E060002882FFF7ADF8641C24B2B442D0
:10FF6000E5DBA86D0021001DA865298270BDA86D84
:10FF70000C30A86570BD2DE9FF5F6B4F7879C00725
:10FF800051D0FEF73CFE6B4D35F8108005EB40007C
:10FF9000B0F80290B0F804A0FEF731FE35F810B0CA
:10FFA00005EB40004188019180880090FEF727FE14
:10FFB0000446FEF724FEFF213970DFF868C15C4F6C
:10FFC0000CEBD00100F0070E08370A7817F80E3056
:10FFD0001A400A70431C0CEBD302167803F0070397
:10FFE0000393FB5C801C1E400CEBD00316701E7844
:10FFF00000F007000290385C06401E7035F81400CF
:020000040801F1
:100000004B4D404511D84B4E06EB440CBCF80260FA
:100010004E450AD8BCF80460564506D2087815F853
:100020000E2010430870BDE8FF9FDFF808C140456F
:1000300015D30CEB44067188494510D351450ED3B6
:1000400058450CD8019FB94209D8B188009EB142E9
:1000500005D803991078695C08431070E3E75845A8
:10006000E1D30CEB4400428801998A42DBD38188BA
:1000700000988142D7D902991878695C08431870B2
:10008000D1E72DE9FC5F284C294F6079254EC00748
:100090005DD0FFF78FFE0190FFF78CFE8346FFF7E0
:1000A00089FE0090FEF7ABFDFF21217000F00703F1
:1000B00006EBD0049A4607F108012278CB5C1A407F
:1000C0002270421C06EBD20502F0070291462B7803
:1000D0008A5C801C06EBD00613402B7000F00700F2
:1000E00080463278085C02403270DDE9001003F08F
:1000F000DFFE06D2207817F80A1008432070BDE80A
:10010000FC9FDDE9001003F0F9FD15D85946009871
:1001100003F0F4FD10D8287817F809100843287068
:10012000EDE700000010002030000020003000202B
:10013000EC5F0008001000205846009903F0DEFD37
:10014000DDD2307817F8081008433070D7E7A06D7B
:100150002030A065D3E72DE9F047FB4D6879C00753
:1001600053D0FFF796FB8146FFF793FB8046FFF7DE
:1001700090FB0446FEF743FDFF212970C117F34BA6
:1001800000EB517503EBE50125F00705DFF8C0C36F
:10019000A0EB050E0A781EF80C50471C2A400A7086
:1001A000421CD51702EB557603EBE60226F0070654
:1001B000BE1B157816F80C703D401570851CEF17A6
:1001C00005EB577503EBE503801C25F00705401B85
:1001D0001F7810F80C502F401F70ACF10805A14596
:1001E00005DD08781EF805201043087087E64445B1
:1001F00004DC1078715D0843107080E6A045F5DAE4
:100200001978405D0143197079E6A86D2030A86522
:1002100075E62DE9F047CC4D6879C00756D0FFF759
:10022000BBF88246FFF7B8F88046FFF7B5F80446FA
:10023000FEF7E5FC01B2FF202870C817C34A01EBA6
:10024000507302EBE30023F00703CE1AC04BB14614
:100250000578F65C864635400570481CC51700EBEE
:10026000557602EBE6074D1C26F00706AE1B97F805
:1002700000C0F55C881C0CEA050CC51700EB557036
:1002800002EBE00287F800C0891C20F00700081A82
:100290001578C15C0D401570A3F10801A24507DD7A
:1002A0009EF8002019F801100A438EF8002026E677
:1002B000444504DC3878715C084338701FE6A0457B
:1002C000F5DA1378405C0343137018E6A86D10301C
:1002D000A86514E62DE9F84FDFF86C8298F8050060
:1002E000C00771D0FFF758F885B2FFF755F886B20E
:1002F000FFF752F887B2FEF782FC0446FEF77FFC58
:10030000FF21DFF848E288F800100EEBD00C9CF8D3
:10031000002000F007018E4B0091595CE0460A4036
:100320008CF80020411C0EEBD10C01F007018B462C
:100330009CF80020595C801C0A400EEBD0018CF820
:10034000002000F0070082460A78185CDFF804E21B
:1003500002400A703EF81400A3F10809A8420FD821
:100360000EEB44025388B3420AD89288BA4207D2AD
:10037000009998F8000019F801100843414620E060
:10038000A84210D10EEB44035A88B2420BD19A888E
:10039000BA4208D19CF8000019F80B1008438CF8F9
:1003A0000000BDE8F88FA842FBD30EEB4400428862
:1003B000B242F6D38088B842F3D9087819F80A20F7
:1003C00010430870EDE7FFE7D8F858101431C8F86B
:1003D0005810E6E72DE9F05F5B4CDFF87491607927
:1003E000DFF86881A9F10809C0075AD0FFF7E2FCDD
:1003F000E062FFF7DFFC2063FEF701FCFF2100B2A3
:100400002170C11700EB517108EBE10521F00701E4
:10041000431A4F499B462A785B5C1A402A70421C5B
:10042000D31702EB537708EBE70627F00707D21B39
:1004300092463378525C1340821C3370D31702EB20
:10044000537308EBE307801C23F00702801A8046F1
:1004500097F800C0405C0CEA000C87F800C0D4E9B3
:100460000B0103F025FD06D228781BF8091008437C
:100470002870BDE8F09FD4E90B0103F0C9FB05D15A
:1004800030781AF8091008433070F2E7D4E90B010C
:1004900003F034FCEDD2387818F8091008433870AE
:1004A000E7E7A06D1830A065E3E72DE9F041264CA1
:1004B0006079C0075DD0FFF7ECF96063FFF7E9F9F9
:1004C000A063FEF79CFBFF2100B22170C11700EB77
:1004D00051721E4901EBE20C22F00702851A1C4AF8
:1004E000A8469CF80030AD5C2B408CF80030431CD3
:1004F000DD1703EB557501EBE50625F00705A3EBCA
:10050000050E37781EF802301F40831CDD1703EB01
:1005100055753770801C25F0070301EBE501C01A03
:100520000F78825C17400F70D4E90D34084A083AFE
:10053000A34211DD9CF8000018F8021040EA010007
:100540008CF8000087E4000030000020001000203C
:10055000F45F00080010002006D130781EF8021069
:1005600040EA0100307076E40B78805C03430B7046
:1005700071E4A06D1830A0656DE42DE9F041FDF740
:10058000FDFFFF4C002854D0FFF783F9E063FFF72D
:1005900080F92064FEF733FBFF2100B22170C11700
:1005A00000EB5172F74901EBE20C22F00702851AC9
:1005B000F54AA8469CF80030AD5C2B408CF8003022
:1005C000431CDD1703EB557501EBE50625F0070528
:1005D000A3EB050E37781EF802301F40831CDD1791
:1005E00003EB55753770801C25F0070301EBE5011F
:1005F000C01A0F78825C17400F70D4E90F34E24ABA
:10060000083AA34208DD9CF8000018F8021040EAFE
:1006100001008CF800001EE406D130781EF80210AC
:1006200040EA0100307016E40B78805C03430B70E5
:1006300011E4A06D1830A0650DE42DE9F047D04C11
:100640006079C0074CD0FEF7A7FE8046FEF7A4FEF7
:100650008146FEF7D4FAFF21217000B2C117C94CC0
:1006600000EB517104EBE10221F00701A0EB010C5A
:10067000C54913781CF80150461C2B401370431CCD
:10068000DD1703EB557304EBE30723F00703F31ABD
:100690003D785E5C35403D70851CEE1705EB567568
:1006A00004EBE504801C25F00705451B2678685CF3
:1006B000083906402670C84506DD10781CF8011080
:1006C00040EA010010701AE405D13878595C40EA1C
:1006D0000100387013E42078695C084320700EE450
:1006E000A06D0C30A0650AE42DE9F047FDF746FF48
:1006F000A34C00284CD0FEF74FFE8046FEF74CFE80
:100700008146FEF77CFAFF21217000B2C1179D4C93
:1007100000EB517104EBE10221F00701A0EB010CA9
:10072000994913781CF80150461C2B401370431C48
:10073000DD1703EB557304EBE30723F00703F31A0C
:100740003D785E5C35403D70851CEE1705EB5675B7
:1007500004EBE504801C25F00705451B2678685C42
:10076000083906402670C84506DD10781CF80110CF
:1007700040EA0100107039E505D13878595C40EA4B
:100780000100387032E52078695C084320702DE55F
:10079000A06D0C30A06529E570B5794C7B4DA06D3E
:1007A0002844C0F34F0001F079FE00286079784AB0
:1007B0004FEAC0701DD170B3A06D41194810C31726
:1007C00000EB537002EBE00220F00700C0EB610089
:1007D0006D4913780839405C03431370FFF759F8EB
:1007E000A16D0839801CA1656066BDE87040FEF708
:1007F0005FBB80B9A06D41194810C31700EB53705F
:1008000002EBE00220F00700C0EB61005E491378C4
:10081000405C03401370A06D0830A06570BD2DE9E9
:10082000F047574C6079C0074FD0FEF705FA804675
:10083000A06DA146001DA065FEF7AEFD85B2207833
:100840004FF0000AFF2811D1002407E038F9140006
:1008500004F10104861947EBE077A4B2AC42F5D36A
:10086000D9F858000838C9F858001FE0D9F85810CE
:1008700001241FFA88F608395746C846C9F85810A7
:100880000FE000BFD8F85810091FC8F85810210110
:10089000A8F81010FEF7D0F986194AEB0707641C78
:1008A000A4B2AC42EED3FF2188F800102A4653468A
:1008B00039463046F4F760F94C46C9F86400FEF753
:1008C000F9FBA06D001DA06590E4A06D0C30FAE767
:1008D0002DE9F0412A494A790846806DD2077DD03A
:1008E0008846C865FEF7D5FFC11700EB117222F0EC
:1008F0000F03A0EB030E1211D31702EB137323F0B7
:100900000F03A2EB030C00EB11621212D31702EBE0
:10091000137323F00F03D31A00EB11521213D417E1
:1009200002EB147424F00F0400EB1140141B0114AB
:10093000CA1701EB127020F00F050011C61700EB6B
:10094000167626F00F06861B01EB12604D1B001277
:1009500001EB1251C717091300EB1777CA1727F0DD
:100960000F0701EB1272C01B22F00F02891A094A0D
:10097000514343F60952504301EB80100CE0000054
:100980003000002000100020F45F0008A49FFFF753
:10099000CD0700208096980040F635414E4340F246
:1009A00071214D4300EB461004EB440100EB0510B0
:1009B000C1EBC41100EBC10003EBC30101EB031158
:1009C00000EB81000CEB8C0100EB410000EB0E0111
:1009D000C8F86410BDE8F041FEF76ABA10308865C7
:1009E000B0E570B5FEF7D8FC0546FEF708F90446F9
:1009F000FEF7D2FCFA4901EB400131F8022C2A4003
:100A0000002101E0491CC9B28142FBDB521E0120DA
:100A1000F449904021F8140070BD2DE9FF47F04FD4
:100A20000025903F7879DFF8C083F04CF04EC00786
:100A30006ED0FEF7B1FC8146FEF7AEFCBA6D32F81F
:100A4000041BC9B2B970BA65E64AB2F8182F8242DF
:100A500005DB94F8E32142F0200284F8E321002929
:100A600054D194F8F211890750D4317800294DD12E
:100A700014F8A01F41F00101217004F24314217801
:100A800001F0DF01217001213170DA49088009EBA2
:100A9000C900D949000191FBF0F64FF40070ADF8A0
:100AA000000003208DF8020010208DF80300761E50
:100AB0006946D248F0F73FFA01210220F0F787FC9F
:100AC00047464046F0F74AFD4720ADF80400ADF830
:100AD0000860ADF80A50ADF8065001A93846F0F7A5
:100AE000D5FD01213846F1F767FA01221146384653
:100AF000F1F77FF801213846F1F766F8012102206D
:100B0000F0F765FCE07B40F00800E073BDE8FF878C
:100B1000B86D30F8081F00F1040011F0FF01B97042
:100B2000B865F3D130780128F0D1B548F1F74CF829
:100B3000002147464046F1F747F801213846F1F7D2
:100B40003BFA002201213846F1F753F8357014F8CA
:100B5000A00F00F0FE00207094F8520100F0F700A2
:100B600084F85201D2E72DE9F0419D4CA54F903C0D
:100B7000A06D3844C0F34F0001F090FCA24DD0B1FD
:100B8000607940006071A06D008820F4504001F051
:100B900093FCF0BBA06DC1194810C21700EB527056
:100BA00005EBE00220F00700C0EB610097491378E5
:100BB000405C034032E0954E207B083E012860797E
:100BC0004FEA40006071A06D008820F450400DD1C4
:100BD00001F072FCE8B1208C844901EBD00100F0F7
:100BE00007000978305C014219D002E001F064FC92
:100BF00078B1607940F001006071A06DC1194810B2
:100C0000C21700EB527005EBE002137820F00700EA
:100C100000E004E0C0EB6100805D03431370A06D51
:100C2000801CA0658EE42DE9F0416D4C754F903C21
:100C3000A06D3844C0F34F0001F030FC734E724D8C
:100C4000083EA0B3207B012860794FEA4000607124
:100C5000A06D008820F4504011D101F02DFC38BB6C
:100C6000208C624901EBD00100F007000978305C6C
:100C700001423AD0607940F00100607125E001F056
:100C80001BFCA8B9607940F001006071A06DC1192A
:100C90004810C21700EB527005EBE00220F007008D
:100CA000C0EB610059491378405C03401CE000E050
:100CB0001BE06079400000F0FE006071A06D0088CC
:100CC00020F4504001F0F8FB78B1A06DC119481034
:100CD000C21700EB527005EBE00220F00700C0EBFA
:100CE00061001378805D03431370A06D801CA065C4
:100CF00028E42DE9F0413A4D424F903DA86D38442B
:100D0000C0F34F0001F0CAFB3F4EC0B1A86D0024F4
:100D1000008820F4504001F0CFFB50BBA86DC119F2
:100D20004810C21700EB527006EBE00220F00700FB
:100D3000C0EB610035491378405C034018E0A86DB2
:100D4000008820F4504001F0B7FB98B1A86D012451
:100D5000C1194810C21700EB527006EBE00220F0F8
:100D60000700C0EB6100294913780839405C034350
:100D7000137000E000246879C10704D0012C02D16F
:100D800040F0010001E000F0FE006871A86D801CD9
:100D9000A86540E42DE9F041114D1A4F903DA86D32
:100DA0003844C0F34F0001F079FB174E80B3A86DB3
:100DB000008820F4504001F07FFB50BBA86D012457
:100DC000C1194810C21700EB527006EBE00220F088
:100DD0000700C0EB61000D491378405C034033E02D
:100DE000C00000200010002000040040001000207F
:100DF000F1000020F200002000A24A04001001408F
:100E0000000C0040A49FFFF7CD070020F45F00080E
:100E100002E0FFE7002418E0A86D0024008820F419
:100E2000504001F049FB80B1A86DC1194810C217AC
:100E300000EB527006EBE00220F00700C0EB61000F
:100E4000FF491378405C034313706879C10704D0ED
:100E5000012C02D140F0010001E000F0FE006871B9
:100E6000A86D801CA865BBE52DE9F041F54DF64F56
:100E7000A86D3844C0F34F0001F010FBF34EC8B129
:100E8000A86D0024008820F4504001F015FB50BBF1
:100E9000A86DC1194810C21700EB527006EBE002B2
:100EA00020F00700C0EB6100E54913780831405C91
:100EB000034017E0A86D008820F4504001F0FCFAD0
:100EC00090B1A86D0124C1194810C21700EB5270EF
:100ED00006EBE00220F00700C0EB6100D849137870
:100EE000405C0343137000E000246879C10701D11E
:100EF000012C02D140F0010001E000F0FE00687119
:100F0000A86D801CA8656BE52DE9F041CD4DCE4F55
:100F1000A86D3844C0F34F0001F0C0FACB4ED8B1F1
:100F2000A86D008820F4504001F0C6FA90B9A86D71
:100F30000124C1194810C21700EB527006EBE00201
:100F400020F00700C0EB6100BD4913780831405C18
:100F5000034019E0002418E0A86D0024008820F464
:100F6000504001F0A9FA80B1A86DC1194810C2170C
:100F700000EB527006EBE00220F00700C0EB6100CE
:100F8000AF491378405C034313706879C10701D1FE
:100F9000012C02D140F0010001E020F00100687155
:100FA000A86D801CA8651BE5A64A8023916D891C4D
:100FB00091650988B3EB112F05D1A549400851F877
:100FC0002000801C90657047F0B59E4E8022B56D64
:100FD000AD1CB5652988B2EB112F19D19D4A3E2170
:100FE000A2F5017432F8113002EB41077B8054F80E
:100FF000213004EB8107491E7B6011F0FF01F1D124
:101000007179118092494008256051F82000B0653F
:10101000F0BD10B58B4CA06D008820F45040FDF75A
:10102000E6FBA06D801CA06510BD10B5854CA06DC1
:10103000008820F4504001F063FAA06D801CA06588
:1010400010BD10B57F4CA06D008820F45040FDF716
:1010500085FBA06D801CA06510BD10B5794CA06DFE
:10106000008820F45040FDF7D7FAA06D801CA065E1
:1010700010BD10B5734CA06D008820F45040FDF7F2
:10108000F0FAA06D801CA06510BD00B56D4B986D89
:10109000008820F45040FDF70AFB986D801C98658D
:1010A00000BD10B5674CA06D008820F45040FDF7DE
:1010B00013FBA06D801CA06510BD10B5614CA06D28
:1010C000008820F45040FDF71CFBA06D801CA0653B
:1010D00010BD10B55B4CA06D008820F45040FDF7AA
:1010E00026FBA06D801CA06510BD2DE9F043554D79
:1010F000DFF864E1D5F858C001243CF8020BC5F8CC
:1011000058C0BCF80010C0B200EB012082B2EA83E4
:10111000287ADFF82C8101090EEB410300F00F0162
:101120004E4E8C4000F56067DFF8149108F1080816
:1011300003F59C6307F0070106EBD706C8282BD3FD
:101140003CF8027F0CF1020C02EB0742C5F858C0D4
:10115000BCF8007002EB076297B2414AEF8302EBE2
:101160008002A5B21468BC4204DA1B889D4301D0FA
:10117000641C1460BC4204DA327818F801100A408A
:1011800003E0327819F801100A433270BDE8F043E9
:1011900000F51C50FDF7E2BA0EEB400707F520679B
:1011A000AF643D88A4B2954204D21B889C4301D011
:1011B0006D1C3D803B889342E3D2DDE72DE9F04191
:1011C000204D254CE88B224604EB400000F50050F2
:1011D0000088E883287A0123010902EB410200F02C
:1011E0000F01DFF85CE01D4E8B4000F56067DFF813
:1011F00050800EF1080E02F59C6207F0070106EB25
:10120000D706C8283BD3EF8B1FFA83FC04EB4704B7
:1012100004F50054648807EB0444A7B2104CEF8334
:1012200004EB80042368BB4205DA12883CEA020C16
:1012300001D05B1C2360EA6C1288BA42327811E05C
:10124000EC5F000830000020A49FFFF7CD070020CE
:10125000240100202C050020001000200010002098
:10126000E018002003D21EF801100A4002E018F82E
:1012700001100A433270A96D091DA9651AE004EB3B
:10128000400404F52064EC649FB22388ED8BAB42EC
:1012900004D21288974301D05B1C23802288AA4283
:1012A000327803D81EF801100A4002E018F8011045
:1012B0000A433270BDE8F04100F51C50FDF74EBA0C
:1012C000F0B4FA4BFB4A9C6DF94F34F8020B9C6565
:1012D0002188C0B200EB012085B2DD83187AA7F126
:1012E000080C00F5606102EBD102167801F00701ED
:1012F000C82818D3241D9C652488002505EB0464A8
:10130000A4B2DC83EC4B53F82030A34202DA795CC0
:101310000E4002E01CF801100E431670F0BC00F500
:101320001C50FDF71BBAE54C04EB400404F52064A7
:101330001C652388AB42EDD2E9E7F0B4DB4DDF4E0C
:101340002946C98B287A06EB410101F500510C882A
:1013500000F56061D74B0A46D54F03EBD1031978EE
:10136000A7F1080C02F00702C828EC8319D3EC8B14
:1013700006EB440606F50056768804EB0644A4B254
:10138000CD4EEC8356F82060A64202DABA5C1140DA
:1013900002E01CF8022011431970A96D091DA9650E
:1013A0000FE006EB400404F520646C652488ED8BA7
:1013B000AC4202D2BA5C114002E01CF80220114398
:1013C0001970F0BC00F51C50FDF7C8B92DE9F041CB
:1013D000B64C40F20117A06D214630F8023B88263A
:1013E000497904F16805A3F20112BB427CD07FDC8D
:1013F0003D2B7BD023DCA3F102033B2B77D2DFE82C
:1014000003F0E7E6E5E7E6E5E4E37676E2E176E0B9
:10141000DF76DE76DD76767676767676E0767676CA
:1014200076767676DCDBDAD9D8D7D676D5D4D3768D
:10143000D2D1D0CFCECDCCCBCAC9C8C7C600512BD4
:1014400074D00FDCA3F13E03132BD7D2DFE803F0F7
:10145000F3F2F1F0EFEEEDECEBEAE9E8E7E6E5E4D4
:10146000E3E2E100762B7ED01FDC6A2B7CD00CDC23
:10147000522B7AD0532B79D0602B78D0622B36D177
:10148000A065BDE8F041FFF7ACBA702B70D0712BAE
:101490006FD0722B6ED0732BF1D1A065C9076AD0C3
:1014A000FEF7F7F902F010FC54E0C02B64D00CDC1E
:1014B000782B62D07A2B61D0822B60D0942BDED136
:1014C000A065BDE8F04101F034BAED2B58D0EE2B09
:1014D00057D0F12BD3D1A065C907E0D0FEF76AFC45
:1014E00002F0C6FB606636E0FBE301E071E232E148
:1014F000D42A47D047DC652A46D046DC352A45D079
:101500002DDC112A7ED012DC022A7CD0042A7BD06A
:10151000062A7AD00E2AB2D1A065C907BFD0FEF73D
:1015200049FC02F0DBF9F4F7B9F811E04CE3122AB8
:101530006CD0142A6BD0162A6AD0182A9FD1A065C5
:10154000C907ACD0FEF736FC02F0C8F9F4F7D0F8C2
:10155000F4F708F92860BDE8F04101F06AB8552AAF
:101560006AD043DC35E08AE35FE337E349E357E3DE
:1015700060E36BE376E306E2A4E38BE38FE39CE3B3
:10158000A5E3A9E3F2E389E0F1E35BE0F0E311E234
:1015900005E2F9E1EBE1E0E1DAE1D4E1CEE1C8E135
:1015A000B6E1A9E1A3E19DE197E18EE185E17FE16B
:1015B00078E171E16BE165E15FE154E139E123E15B
:1015C0000DE1DDE006E1F3E0EDE0E7E0E2E0DDE0A3
:1015D000D8E0362A74D04F2A73D0512A72D0532AB9
:1015E00099D1A065BDE8F04101F074B95B2A6AD0D9
:1015F0005D2A69D0632A68D0642A8CD1A065C907A6
:101600008CD01AE0A1E378E393E383E3A6E3B0E3AD
:10161000BAE3CFE2BCE2A9E29EE28EE286E277E2A2
:101620006AE25FE250E242E237E22CE220E211E2BB
:1016300002E2F0E1EAE1D1E1CDE3FDF7ADFEFCF736
:1016400081FF48E1CB2A7ED01BDCC42A7CD00BDC96
:10165000662A7AD0C12A79D0C22A78D0C32ABFD1CB
:10166000A065BDE8F04110E5C52A71D0C62A70D04A
:10167000C92A6FD0CA2AB3D1A065BDE8F041FFF7EF
:10168000D2BACC3A082A66D2DFE812F0F403F903A2
:10169000FE03030408040D0412041704F02A70D09A
:1016A0002FDCA2F1D702192AEDD20FE03000002082
:1016B000F45F000800100020E01800200010002057
:1016C00076E37EE382E38BE38FE393E3DFE812F0DC
:1016D000FF0304040904210426042B04080508055B
:1016E000300438044204490454045B040805080526
:1016F00065046C04760482048D04940408050805CE
:10170000A404FC2A7DD010DCA2F1F1020B2ABAD28B
:10171000DFE812F096049F04A604B004E604E60491
:10172000B904C004C904D004D90440F63F73A2F63A
:101730003F719A427BD018DCA2F570620F3A5AD002
:10174000022A6DD008E090E37BE366E36FE373E386
:101750007CE380E384E3F2E3142A69D0152A8AD17A
:10176000A065BDE8F041FEF708BF012979D0022944
:1017700078D0A1F56741BF39F1D1A0650020207371
:1017800011E4F8E3A065BDE8F0415AE4A065BDE8C6
:10179000F0413EE4A065BDE8F04146E4A065BDE847
:1017A000F041FDF7B0B8A065BDE8F041FDF70CB918
:1017B000A0650088010A862908D08E29E0D1C0B230
:1017C00000F0E2FEA06D801CA065D9E7C0B200F079
:1017D000A6FEF7E7A065BDE8F04100F0FBBEA065FE
:1017E000C90710D00088B6EB102FC9D1BDE8F04171
:1017F000C0B2FFF7D9BBA065FCF7C0FE10B1A06D69
:10180000F0E7F1E3A06DFAE1A065C907FBD000881D
:10181000B6EB102FB4D1BDE8F041C0B2FFF7D4BB96
:10182000A065FCF7ABFE0028ECD0A06DEFE7F6E07A
:101830001EE0F94A10886071A2F501710B683E2024
:10184000C4F8583002EB40035B8822F8103001EBFB
:1018500080035B68441E41F8203014F0FF00F1D192
:101860008EE7F2E0FEE0A065BDE8F041FEF7E5BEE0
:10187000A065BDE8F041FEF737BFA065BDE8F041C7
:10188000FEF713BEA065BDE8F041FEF7C2BCA0653F
:10189000BDE8F041FEF75FBCA065C90772D0FDF757
:1018A0007BFD10E0A065C9076DD0FDF7F2FF12E0E7
:1018B000A065BDE8F04100F0BBBFA065C907EDD051
:1018C000FDF76AFDC04360662CE1A065C907EBD057
:1018D000FDF7DFFFC043606600E1A065BDE8F041B1
:1018E000FEF713BBA065BDE8F04100F075BFA06531
:1018F000BDE8F04100F048BFA065C907CED0FDF7B4
:101900004BFD0546FDF748FD0146A06D08380AE08D
:10191000A065C807A4D0FDF7BCFF0546FDF7B9FFD9
:101920000146A06D10386166A065FDF7C1FA284632
:10193000D1E7A065BDE8F04101F0DBB8A065BDE8E6
:10194000F04101F07CB8A065BDE8F04101F0FAB8C3
:10195000A065BDE8F041FEF7BBBFA065C90772D026
:10196000FDF71AFD0546FDF717FD2844ABE7A06516
:10197000C90769D0E065FDF78CFF0546FDF789FFD3
:101980002844A8E7C3E050E2A065C907E7D0E065B6
:10199000FDF702FD0546FDF7FFFC281A93E7A06559
:1019A000C907E6D0E065FDF774FF0546FDF771FF56
:1019B000281A90E7A065C90745D0E065FDF7ECFC63
:1019C0000446FDF7E9FC0546FDF736F96C43046073
:1019D000D6E6A065BDE8F04101F0DDB8A065C90715
:1019E00070D0E065FDF7D8FC0446FDF7D5FC054650
:1019F000FDF705F994FBF5F201B2884B05FB1240A7
:101A000023F8112003EB41014880B9E6A065BDE849
:101A1000F04101F0E9B8A065C90777D005E0A065FD
:101A2000FCF7ACFD00283FF4EDAEFDF7B5FCA16D71
:101A3000091F401CA16546E7A065C90767D0FDF7EF
:101A400028FF401C1AE03DE0A1E0A065BDE8F041A0
:101A5000FEF7A2BEA065C907DFD000BFFDF79CFC62
:101A6000401E5BE0A065FCF789FD0028F6D1C9E6C1
:101A7000A065C907E2D0FDF70CFF401E6066A06DAF
:101A80000838A0652AE0A065C9071BD0FDF784FCD3
:101A90000546FDF781FC054012E0A065C90776D038
:101AA000FDF7F7FE0546FDF7F4FE054015E0A065DD
:101AB000C90707D0FDF770FC0546FDF76DFC05432F
:101AC00065662FE00C307FE6A065C907E7D0FDF71B
:101AD000E0FE0546FDF7DDFE05436566BDE8F04125
:101AE000FDF7E6B9A065C907ECD0FDF755FC054642
:101AF000FDF752FC4540E3E7A065C907CFD0FDF7ED
:101B0000C8FE0546FDF7C5FE4540E6E776E082E102
:101B1000A065C90773D0FDF73FFC40426066A06D29
:101B2000001FA065BDE8F041FDF7C4BAA065C90774
:101B300084D0FDF7AEFE4042A0E7A065C90799D06A
:101B4000FDF72AFC85B2FDF727FC80B225FA00F1EB
:101B5000C0F11000854017E0A065C8073FF435AE1E
:101B6000FDF797FE0546FDF794FE1AE0A065C9074C
:101B7000DED0FDF711FC85B2FDF70EFC80B205FA50
:101B800000F1C0F11000C5402943616630E0CEE0AD
:101B9000A065C807E2D0FDF77CFE0546FDF779FE9B
:101BA0004042C5416566A06D1038A065FDF780F91B
:101BB000A06D30E1A065C907FBD0FDF7EDFB85B254
:101BC000FDF7EAFBC54012E0A065C807C6D0FDF7E7
:101BD00060FE0546FDF75DFEC540E3E7A065C90769
:101BE000E7D0FDF7D9FB85B2FDF7D6FB85406566EA
:101BF000A06D0838A065FDF75DFA03E6FFE7001D5C
:101C0000E2E5A065C807A9D0FDF743FE0546FDF74C
:101C100040FE8540C6E700002C0500200010002093
:101C2000A065BDE8F04100F082BDA065BDE8F041CF
:101C3000FEF7F5BDA065C80790D0FDF7ADFBF4F742
:101C4000A7F9F3F72BFDF4F769F9E2E0A065C807FF
:101C500084D0FDF71EFEF4F79BF9F3F71FFDF4F7B0
:101C60005DF930E6A065C907A3D0FDF795FB02F04A
:101C70002BF8286000F0DDFCA06D001FA4E5FC4DF2
:101C8000A065C90703D0FDF787FB287078E50A2116
:101C90002970B4E7A065BDE8F041FEF7DEB8A065A5
:101CA000FDF7F7FD0546FDF7F4FDA84276D1607912
:101CB000C10773D0ADE1607162E5A065BDE8F04198
:101CC000FEF7ABBEA065BDE8F04100F0C4BCA06566
:101CD000BDE8F041FEF77EBBA065BDE8F041FEF730
:101CE000D0B9A065C90722D0FEF764F80446FEF714
:101CF00061F8214601F01AFE2CE4A065C90716D050
:101D0000FEF758F80446FEF755F80146204602F063
:101D100005F91FE4A065C90709D0FEF74BF8044692
:101D2000FEF748F80146204601F080FE12E4183024
:101D30004AE5A065C907FAD0FEF73CF80446FEF76D
:101D400039F8214602F00AF804E4A065C90762D018
:101D5000FEF730F801F08CFF80B2DFE6A065C9071E
:101D600063D0FEF727F801F083FFB4E5AAE049E06D
:101D700015E0A065C90758D0FEF71CF801F0AEFDCC
:101D8000F3F73CFCFFF7E4BBA065C9074DD0FEF7B5
:101D900011F801F0A3FDF3F7E3FBF3E735E1A065EC
:101DA000C90738D0FDF7F8FA011241EA0020B5E67C
:101DB000A065C8073FF409ADFDF76BFD4FEA304061
:101DC0005CE6A065BDE8F041FEF784BAA065BDE819
:101DD000F041FEF7D0B8A065BDE8F04100F00BBEC1
:101DE000A065BDE8F04100F0C5BDA065BDE8F041CB
:101DF00000F0E2BDA065C9070DD0FDF7CDFAFCF7F4
:101E0000A1FB06E0A065C90705D0FDF7C5FAFCF700
:101E1000A7FB80B257E50830D6E4A065C90704D017
:101E2000FDF7BAFAFCF79CFB55E51030CCE4A06551
:101E3000BDE8F041FFF711B9A065BDE8F041FFF73B
:101E400018B9A065BDE8F041FFF72BB9A065BDE862
:101E5000F041FFF732B9A065BDE8F041FFF739B9AD
:101E6000A065BDE8F041FEF77EBEA065BDE8F0418B
:101E7000FEF73FBFA065BDE8F041FEF78BBFA06550
:101E8000BDE8F041FEF7F0BFA065BDE8F041FFF707
:101E90003BB8A065BDE8F04100F0F5BEA065BDE827
:101EA000F04100F0CCBEA065BDE8F04100F042BFBB
:101EB000A065BDE8F04100F00ABFA065BDE8F041B3
:101EC00000F081BFA065BDE8F04100F058BFA065FB
:101ED000BDE8F04101F02BB8A065BDE8F04101F08C
:101EE00002B8A065FDF758FA0546FDF755FA217BC3
:101EF000012904D185427FF768AC6079EDE0617912
:101F00004906090E617185423FF75FAC41F001005F
:101F1000D1E6A065BDE8F04100F079BFA065BDE85D
:101F2000F04100F0BCBFA065BDE8F04100F093BFF8
:101F3000A065FDF731FA0546FDF72EFA06E0CFE081
:101F4000A065FDF7A6FC0546FDF7A3FC85423FF41E
:101F5000AEAE5AE0A065FDF71FFA0546FDF71CFA84
:101F600005E0A065FDF795FC0546FDF792FC85426E
:101F70003FF79DAE49E05AE0A065FDF70DFA054632
:101F8000FDF70AFA05E0A065FDF783FC0546FDF7BD
:101F900080FC8542FFF68BAE37E0A065FDF7FCF9CB
:101FA0000546FDF7F9F905E0A065FDF772FC054669
:101FB000FDF76FFC85427FF47AAE26E0A065FDF761
:101FC000EBF90546FDF7E8F9854296DC6079C10733
:101FD00093D01EE0A065FDF75CFC0546FDF759FCBB
:101FE00085427FF764AE10E033E0A065FDF7D4F9D9
:101FF0000546FDF7D1F905E0A065FDF74AFC054669
:10200000FDF747FC8542BFF652AE607920F0010033
:1020100051E640F001004EE6A065FDF7BDF905462A
:10202000FDF7BAF909E06079C10756D053E0A06521
:10203000FDF72FFC0546FDF72CFC8542F3D14AE065
:10204000A065FDF7A9F90546FDF7A6F98542EADD89
:1020500041E0A065FDF71DFC0546FDF71AFC38E0E0
:10206000A065FDF799F90546FDF796F908E000002F
:10207000F0000020A065FDF70CFC0546FDF709FC0B
:102080008542D0DA27E0A065FDF786F90546FDF721
:1020900083F905E0A065FDF7FCFB0546FDF7F9FBBC
:1020A0008542C0D017E0A065FDF776F90546FDF73B
:1020B00073F905E0A065FDF7ECFB0546FDF7E9FBCC
:1020C0008542B0DC07E0A065FDF766F90546FDF73F
:1020D00063F98542A7DB60799BE700F0FE00EAE543
:1020E000022140F64170FCF781FAFFF76BBB70B537
:1020F000F84EF7480021F84CB02343F67F65B065F1
:102100000288B3EB122F02D1D2B244F82200491C4C
:10211000801C89B2A942F3D3B06570BDEF4900209D
:10212000488008807047EA4910B5891EE94B0020B5
:1021300043F67E629965401C31F8024F80B20F2C45
:1021400001D09042F7D3996510BD2DE9F047E448DE
:102150000068E24FDFF88CC3DFF88C93E34AE44B6E
:10216000DC4C0126A03F0025002870D020790921F1
:10217000012803D1257183F8E01103E093F8E00111
:10218000092865D198468A46C2F8A051E07A58B924
:10219000FFF7ADFFE672FFF7C6FF43F67E618842A8
:1021A00002D988F8E0A12CE1E07840B908F5F07098
:1021B000017841F00401C9B201F0F7010170C4488F
:1021C000A0659CF8000008B9F0F728FEA16D08880A
:1021D000020A5E2A72D032DC5E2A70D2DFE802F098
:1021E000F06F6F6F6F6FA36F6F6F6F6F6F6FBA6FFF
:1021F0006F6F6F6F6F6F6F6F6F6F6F6F6F6F6F6FEF
:10220000D0D0D0D0D0D0D0D0D0D0D0D0D0D0D0D0CE
:10221000D5D5D5D5D5D5D5D5D5D5D5D5D5D5D5D56E
:10222000DBDBDBDBDBDBDBDBDBDBDBDBDBDBDBDBFE
:10223000E0E0E0E0E0E0E0E0E0E0E0E0E0E07F2AB5
:1022400070D018DCA2F15F02202AC6D201E004E1BE
:10225000EBE0DFE802F0A5AAAAAAAAAAAAAAAAAA5B
:10226000AAAAAAAAAAAAAAAFAFAFAFAFAFAFAFAFA1
:10227000AFAFAFAFAFAFDC2A1FD028DCCC2A0BD07A
:1022800012DCC82AFBD008DCB02A6FD0C52AF6D0F1
:10229000C62AF4D0C72A12D194E0C92AFCD0CA2A8F
:1022A000FAD0CB2AF7D18DE0D82AE5D008DCCD2AA8
:1022B00070D0CF2A6ED0D52AEDD188E070E080E0D2
:1022C000D92A03D0DA2A01D0DB2AE4D17FE0EC2A34
:1022D00009D010DCE82A7FD006DCDD2A77D0DF2A9F
:1022E00075D0E52A6DD177E0E92A75D0EA2A73D056
:1022F000EB2A66D170E0F12A73D006DCED2A6BD0B0
:10230000EF2A69D0F02A79D16BE0F22A69D0F32A5A
:1023100067D0FF2A72D1C0B2FCF7C3FAA06D801C4F
:10232000A06553E746E0E071891CA1650888000AB2
:10233000802804D08628F1D100F04AFEEEE76079CB
:10234000C00702D000F017FEE8E7891CA16500F085
:102350002EFEE3E72072891CA1650888000A802808
:1023600005D08628DAD100F06BFED7E73EE0607931
:10237000C00702D0FEF7B9FED0E7FEF7A1FFCDE718
:10238000C0F30B00FCF748F9C8E7C0F30B00FCF7FB
:1023900068F9C3E716E0C0F30B00FCF788F9BDE766
:1023A000C0F30B00FCF798F9B8E7C0F30B00FCF79B
:1023B000A8F9B3E7C0F30B00FCF7B9F9AEE706E004
:1023C00017E01BE0C0F30B00FCF7C8F9A6E7C0F369
:1023D0000B00FCF70CFAA1E7C0F30B0000F090F83B
:1023E0009CE7C0F30B00FCF743FA97E7891CA16553
:1023F000ECE6C0B21C2804D00F2802D0FEF7E6FF9E
:10240000E4E6B9F80000A7F8180EA7F8160EA7F82A
:10241000140EA9F80050E67098F8E00100F0FB00F7
:1024200040F0080088F8E00134E000F0FE0040F0E1
:10243000020083F8E001A7F8185EE572E570C2F8C3
:10244000A0619CF8000028B9FFF768FEF0F7E6FCF1
:10245000F0F737FE257365731CE0FFF75FFE93F816
:10246000E00100F0FE0040F0020083F8E001A7F870
:10247000185EE572E570C2F8A0618CF80050F0F7C4
:10248000CDFC25736573207920B92671A9F8005019
:10249000F0F717FEA7F8025EBDE8F0871549164A67
:1024A00001EBD00100F007000978105C014201D077
:1024B00001207047002070470D490F4A01EBD00101
:1024C00000F007000978105C014217D00120704726
:1024D0005C6000083000002024010020A0100020D3
:1024E00034012242F5000020E40000200080214257
:1024F00000100020CD070020EC5F00080020E6E778
:10250000FF494979C907E2D0FE49FF4B01EBD001F1
:1025100000F007000A78185C02400A70D7E7F0B5AF
:10252000F749F84F4979F84ECB0700F50C5101F007
:10253000070207EBD10122D000F5C06407EBD403FA
:1025400004F007041D78345D25401D7000F5185314
:102550001C4607EBD30304F007041D78345D2540C7
:102560001D70A6F108040B78A25C1343E74A0B70B8
:1025700002EB4000002100F580500180F0BD08789A
:10258000B25C10400870F0BDF0B4DD4B5979C9075A
:102590001BD0DE49DB4E00F1E004A0F1C80501EBE1
:1025A0004001002704F00702DFF85CC301F5206159
:1025B00006EBD404372D01D821F8027B59620F8035
:1025C00021781CF8022011402170F0BC00F55C500D
:1025D000FCF7C4B8CA4A10B450791146896DC007D7
:1025E00024D031F8020B91650A880023110AC74CE8
:1025F000C0B2862901D0882904D100EB0220C0B2E4
:10260000002105E080290AD100EB0220C0B2E821B8
:1026100001EB5000C0B224F8103010BC704710BC61
:1026200041F6651140F64170FBF7E0BF091D916569
:10263000F3E710B5FCF7E3FAB14AB44968321388FE
:1026400021F8103001EB40005288AD494280886D7E
:10265000001D886510BD2DE9F047A9484079C007E5
:1026600064D0FCF7E9FAB0F80080FCF7E5FAB0F9BD
:102670000090FCF7E1FA0546FCF7DEFAB5F9002018
:10268000B5F90830B5F9187092FBF3F6B5F90E30CC
:10269000B5F806E006FB03762F8AB5F90AC0B5F94E
:1026A0000C10DB1B334403FB0EF3AB836E8A05F186
:1026B0000E04A6EB0803EB81B5F90430B5F914500C
:1026C000C3F101065D4306FB09530CFB012291FB9C
:1026D000F2F51BB2A3800CFB01FCB4F908609CFB73
:1026E000F2F13344B4F90660B4F90C20764203EBFE
:1026F00046035D4301FB02516181B0F90010B4F95A
:102700000E20114447F6FE72914201DD511C04E097
:102710007F4A914201DC028000E001806089A08153
:10272000E0882081A088E08020886080B4E670B5D1
:10273000734D6879C00723D0FCF761FA0446FCF7B3
:102740005EFA01462878B0B96E4B6F4D0AE000BFC3
:1027500003EBD40004F007060278AE5D3240641C3F
:102760000270A4B28C42F3D970BD00BF20F81420CF
:10277000641CA4B201E0654800228C42F6D970BD09
:10278000A86D0830A86570BD70B55D4D6879C0074B
:1027900021D0FDF77EF86866FCF78AFBFDF779F833
:1027A00006B2A86D08380124A8650DE0687A0128F2
:1027B00001D1600100E0A0002882A86D0838A8655A
:1027C000FCF776FB641C24B2B442EFDBA86D002159
:1027D000001DA865298270BD70B5494D6879C00794
:1027E00022D0FCF7D9FD6866FCF764FCFCF7D4FD49
:1027F0000646A86D001F0124A8650DE0687A01282F
:1028000001D1200100E060002882A86D001FA865AA
:10281000FCF750FC641C24B2B442EFDBA86D00212D
:10282000001DA865298270BDA86D0C30A86570BD1B
:102830002DE9F04732484179C90747D0FCF7ACFD94
:1028400087B2FCF7A9FD84B2FCF7A6FD86B2FCF7BF
:10285000D6F90546FCF7A0FDDFF8A4E081B20EF141
:10286000740E3EF81400B7FBF0F200FB1272002069
:10287000264F28E0641EA4B23EF81430491E984644
:10288000B2FBF3F389B23EF811C0994603FB0CF397
:1028900037F815C0012C43EA0C039BB227F815301A
:1028A0000DD101290BD1BEF802C002F00F0000FBD0
:1028B0000CF0184327F81500701C80B201E008FBEB
:1028C0001922401C80B2B042D4D3E5E5816D1431A9
:1028D0008165E1E570B50A484079C00728D0FCF76A
:1028E0008EF90546FCF78BF90446FCF788F9074991
:1028F00031F8152031F814301A4421F8102009E07D
:102900003000002000100020F45F000800100020BC
:102910000080FFFF01EB450201EB440355885C8812
:1029200001EB40002C44448091889A8811448180B6
:1029300070BD10B5F8484179C90717D0FCF75FF9A9
:10294000C11700EB5173F54901EBE30223F00703D4
:10295000C31AF3481178185C014204D0F0480830DB
:10296000185C014000E00143117010BD816D091D2C
:10297000816510BD10B5E8484179C90718D0FCF74A
:102980003EF9E849B1F8242E21F81020B1F8222EA2
:1029900001EB4000428001F61A61CA8882808A8871
:1029A000C2804A8802810A8842818989818110BD5A
:1029B000816D091D816510BD1CB5D7484179C907D6
:1029C00015D0FCF71CF9D74C04EB40014A89D3B26F
:1029D0000A89D2B2CDE90023CA8834F81000D3B2F4
:1029E0008A884988D2B2C9B2F1F73DFE1CBD816D1B
:1029F000091D81651CBD70B5C7484079C0071DD051
:102A0000FCF7FDF80546FCF7FAF80446FCF7F7F882
:102A1000C44931F8152031F81430D21A21F81020A9
:102A200001EB450201EB440355885C8801EB400053
:102A30002C1B448091889A88891A818070BD2DE969
:102A4000F041B5494A790846806DD2074DD0884695
:102A5000C865FCF71EFF0A2190FBF1F292FBF1F32F
:102A600001FB120E01FB1323642290FBF2F292FB96
:102A7000F1F401FB142C4FF47A7290FBF2F292FB0A
:102A8000F1F401FB142442F2107290FBF2F292FB7B
:102A9000F1F501FB1525A44A90FBF2F292FBF1F649
:102AA00001FB1626A14A90FBF2F292FBF1F701FB23
:102AB00017229F4F90FBF7F090FBF1F701FB1700F7
:102AC00002EB0010000600EB065000EB054000EBA7
:102AD000043000EB0C2000EB031000EB0E01C8F8F3
:102AE0006410BDE8F041FCF7E3B910308865BDE83B
:102AF000F08110B5884C61792046806DC9071ED0E1
:102B0000E065FCF749FC4FF47A7390FBF3F103FBAB
:102B100011000A03642390FBF3F103FB110042EA66
:102B200001220A2390FBF3F142EA011203FB110098
:102B300012B202436266BDE81040FCF7BBBA08302F
:102B4000A06510BD10B5744C61792046806DC90731
:102B50001ED0E065FCF720FCC0F303324FF47A711D
:102B60004A43C0F3032101EBC10303EB011102EB64
:102B70008102C0F3031101EB810102EB410100F07E
:102B80000F00084400B26066BDE81040FCF792BA3E
:102B90000830A06510BD70B55F4D6879C0071FD0C3
:102BA000FCF777FE0446FCF774FE4443E11705F199
:102BB0008000C0E90241FCF722F8A96D594A091DBD
:102BC000A96505F1880100B20B8822F810304B8806
:102BD00002EB400043808A888280C988C18070BD32
:102BE000A86D1830A86570BD70B54B4D6879C007E9
:102BF00021D0FCF74EFE04B2FCF74BFE00B294FB72
:102C0000F0F105F16C0600FB1140341D31602060CD
:102C1000FBF7F5FFA96D00B2091DA965414932888E
:102C200021F81020728801EB4000428021888180C9
:102C30006188C18070BDA86D1830A86570BD10B5E1
:102C4000FCF727FE0446FCF724FE334A117B0129DA
:102C500051794FEA41614FEA1161517110D18442BB
:102C60000DD1108C2D4B2E4C03EBD00300F0070040
:102C70001B78205C034202D041F00100507110BD6E
:102C80008442F9D010BD10B5FCF786FB0446FCF772
:102C900083FB214A117B012951794FEA41614FEAB7
:102CA0001161517110D184420DD1108C1B4B1C4C01
:102CB00003EBD00300F007001B78205C034202D036
:102CC00041F00100507110BD8442F9D010BD10B523
:102CD000FCF7DFFD0446FCF7DCFD0F4A117B012900
:102CE00051794FEA41614FEA1161517110D184422B
:102CF0000DDD108C094B0A4C03EBD00300F00700EC
:102D00001B78205C034202D041F00100507110BDDD
:102D10008442F9DB10BD00003000002000100020CC
:102D2000EC5F000800100020A086010040420F0068
:102D30008096980010B5FCF72FFB0446FCF72CFB9F
:102D4000D04A117B012951794FEA41614FEA116163
:102D5000517111D18442DDDD108CCB4BCB4C03EB98
:102D6000D00300F007001B78205C0342D2D000BFE4
:102D700041F001005071CDE78442F9DBCAE710B59C
:102D8000FCF787FD0446FCF784FDBE4A117B012950
:102D900051794FEA41614FEA1161517110D184427A
:102DA000B8DA108CB84BB94C03EBD00300F0070035
:102DB0001B78205C0342ADD041F001005071A9E7BF
:102DC0008442F9DBA6E710B5FCF7E6FA0446FCF707
:102DD000E3FAAC4A117B012951794FEA41614FEA8C
:102DE0001161517110D1844294D1108CA64BA74C23
:102DF00003EBD00300F007001B78205C034289D06E
:102E000041F00100507185E78442F9DB82E710B59B
:102E1000FCF73FFD0446FCF73CFD9A4A117B012973
:102E200051794FEA41614FEA1161517110D18442E9
:102E30000DDC108C944B954C03EBD00300F0070095
:102E40001B78205C034202D041F00100507161E721
:102E50008442F9DD5EE710B5FCF71BFD0446FCF784
:102E600018FD884A117B012951794FEA41614FEAE7
:102E70001161517110D184420DDB108C824B834C57
:102E800003EBD00300F007001B78205C034202D064
:102E900041F0010050713DE78442F9DA3AE710B59C
:102EA000FCF77AFA0446FCF777FA764A117B012997
:102EB00051794FEA41614FEA1161517110D1844259
:102EC0000DDB108C704B714C03EBD00300F007004E
:102ED0001B78205C034202D041F00100507119E7D9
:102EE0008442F9DA16E710B5FCF7D3FC0446FCF788
:102EF000D0FC644A117B012951794FEA41614FEAC4
:102F00001161517110D184420DD0108C5E4B5F4C19
:102F100003EBD00300F007001B78205C034202D0D3
:102F200041F001005071F5E68442F9D1F2E610B5A6
:102F3000FCF732FA0446FCF72FFA524A117B0129BA
:102F400051794FEA41614FEA1161517110D18442C8
:102F50000DD0108C4C4B4D4C03EBD00300F0070010
:102F60001B78205C034202D041F001005071D1E691
:102F70008442F9D1CEE610B5424C454AA06D30F8F6
:102F8000021BA0650088C9B201EB0021A183E07992
:102F900002EB400202F5905262641180EFF7B9FA39
:102FA000E079BDE8104000F5B050FBF7D7BB10B595
:102FB000344CE079EFF7E9FAE07900F5B050FBF72F
:102FC000CDFBE079BDE8104000F5C060FBF7C6BB63
:102FD00010B52C4CA06D30F8021BC1F34601A18343
:102FE000A0650088010A862922D0882906D1A18BF4
:102FF000C0B201EBC01000F57A70A0836079C00701
:103000001BD02349A08B01EB400000F50050028843
:10301000E07901EB400101F58051A1F80022EFF7C2
:1030200078FAE079BDE8104000F5B050FBF796BBA8
:10303000A18BC0B201EBC010DFE7BDE81040B6E7DE
:10304000104A906D30F8021BC1F34601D1839065A0
:103050000088010A86290DD0882906D1D18BC0B2FB
:1030600001EBC01000F57A70D0835079C00706D00C
:10307000FEF7A4B8D18BC0B201EBC010F4E7FEF7A5
:103080005CB900003000002000100020EC5F000858
:103090000010002051EA030C17D41CF5801F58BF04
:1030A000BCF5801F00F10680994218BF704708BF29
:1030B0009042704707D711F5801F58BF13F5801F46
:1030C00019D499427047894270471CF5801F08D572
:1030D000BCF5801FF7D58B4218BF704708BF8242EE
:1030E00070474FF4001C1CEB410F38BF1CEB430F23
:1030F00001D28B427047DFF808C0F2F785BC0000B0
:1031000019001604DFF8B4C170B53CEA111E18BFEF
:103110003CEA131E00F0A68081EA03050CEA111EAA
:103120004EEAD57E1CEA131518BF11EA0C1F00F0F9
:103130008F80AE4421EA4C1123EA4C13AEF17F7E1E
:1031400041F4801143F48013A1FB024CA0FB036502
:10315000361955EB0C05A1FB034C4CF10003A0FB09
:10316000021C16EB0C06654153F10003094218BF1F
:1031700046F001064FF0140CB3F5007F4CF1000C43
:10318000CCF1200425FA0CF203FA04F141EA020121
:1031900005FA04F026FA0CF240EA02006FF003028E
:1031A00042EB2E4216FA04F401EB025585EACE7189
:1031B00015D05FEA440C38BF4FF040440FD308BF2E
:1031C00043F0004350F1000041F1000110EAD37FC9
:1031D0004FF0804420EAD37018BF4FF0404415F000
:1031E000004FDFF8DCC017D415EA0C0F18BF3CEA1B
:1031F000010C11D070BD5FEACE7454BF1CF4000FF7
:103200001CF4800F0ABF4FF080444FF0404410F18F
:10321000010041F10001E2E7BEF1806FA2BFA1F120
:10322000C04144F0130C4CF0805CBDE8704006DAFD
:103230004FF0000001F1C04101F0004170476FF014
:10324000000041EA500181EA10314FF00000704760
:103250004FEACE714FF0000070BD4FEACE714FF0D3
:10326000000070BD4FEA4105B5EB4C1F4FEA430625
:1032700008BF002898BFB6EB4C1F08BF002ABDE866
:103280007040DFF840C031F6ABAEAFF300804FF4D2
:10329000001CBCEB410F98BFBCEB430F0AD84FF0AA
:1032A000000081EA030101F0004141F0FE4141F4D8
:1032B0007001704704494FF0000070470000FF079D
:1032C0000000F07F130000040000F87FDFF888C1E1
:1032D00070B53CEA111418BF3CEA131500F08F805A
:1032E00011F1004F1CEA13150CEA111468BF45F0E8
:1032F000050518BF11EA0C1F00F079802E4621EA5F
:103300004C1123EA4C1341F4801143F48013A5F5CA
:103310008035AC423DDD801A9941A4F5803609D54F
:103320004042C1F1000134BFB1F10101B1F100012E
:1033300085F0010511F4F01F08D011F4801FE8D1C9
:10334000400041EB0101A4F58034F6E721F0004193
:10335000B1FA81F6202E04BFB0FA80FE0EF12006ED
:10336000A6F10B06B6F1200EA4EB06440CD2C6F172
:10337000200E01FA06F120FA0EF641EA0601CEF11E
:10338000200600FA06F003E000FA0EF14FF000000C
:10339000BFE750EA410E23D04FEA244EBEEB254F43
:1033A0000FDB994208BF904204D00AD3520043EB8E
:1033B0000303B0E74FEA1646B6EB144F08BF85F09B
:1033C0000105B4F5803401EB041181EAC57100DB1D
:1033D00070BD01F1C0414FF0000001F0004170BD2F
:1033E0004FEA45714FF0000001F0004170BD1CEA4A
:1033F000131F2BD04FF0000001F0004170BD4FEAC9
:103400004106B6EB4C1F4FEA430E08BF002898BF99
:10341000BEEB4C1F08BF002ABDE87040DFF83CC07F
:1034200031F6DEADAFF300806FEA115C5FEA4C5C11
:103430000ED01CF5001F38BF704750EA410208BF8C
:1034400070474FF0000001F000417047BDE8704048
:103450004FF00000024970470000FF07150000040C
:103460000000F87F4FF0E04C4CF07F6C70B511EA33
:103470000C0F00F078803CEA010E00F07D8011F026
:10348000004F40F087804FEA115C21EA0C5141F473
:1034900080110CF1FD0C5FEA5C0C0CF5C07C02D3D2
:1034A000400041EB01014FF000034FF080424FEA32
:1034B000812141EA90514FEA8020A1F180414FF0F3
:1034C000805E8C1A22BFB4EB0E04214602EB4E0242
:1034D000400041EB01015FEA5E0EF2D171EB0204A4
:1034E00007D3B0F1004574F1000422BF21462846FD
:1034F000521C400041EB01014FF0804EC51A71EBA8
:10350000020408D3B5EB0E0574F1000422BF214676
:10351000284603EB4E03400041EB01014FEA5E0EEB
:10352000BEF1800FEAD151EA000418BF0224980AC4
:103530004FEA92215FEA340440EA825001EB0C51D9
:1035400000D170BD640050F10000244241F100013F
:1035500008BF20F0010070BDDEF5800E50F10000C4
:1035600041F1000170BD50EA013C00D170BD01F095
:1035700000414FF0000070BDBDE8704050EA013CD2
:10358000DFF81CC071F434ADAFF30080094258BFBE
:10359000704701E0BDE870404FF0000001497047FE
:1035A000170000040000F87F10B591EA030F48BF30
:1035B00083F0004332F528A9841A71EB030E07D279
:1035C00012198EF0004E43EB0E03001B61EB0E014F
:1035D000DFF810C24FEA1154A4EB135E1CEA430F4C
:1035E00018BF9CEA445F00F0C58023EA6C03524296
:1035F00021EA0451C3EB6C0338BF5B1EDEF1200CE3
:1036000029D322FA0EFC10EB0C0043FA0EFC41EB1E
:103610000C01CEF1200C03FA0CFC10EB0C0051F164
:103620000001CEF1200C2DD401EB0451BDE8104077
:1036300012FA0CF24FF0120C4CF0804C58BF70474D
:10364000401C1CBFB2F1004F704700280CBF491C42
:1036500020F00100704712EB020C43EB030218BF8D
:103660004FF0010C4CEA4202AEF1200EDEF11E0CCE
:1036700063D943FA0EFC10EB0C0051F1FF31CEF18F
:103680001E0CD1D50CF1010C12FA0CFC404141EB9F
:10369000010101EB445E5FEA5E5E10D901EB04516B
:1036A000BDE8104010EBDC7038BFBCF1004F18BF14
:1036B000704700280CBF491C20F0010070473FD222
:1036C00011F5001108BF002801D1BDE810403FD01E
:1036D0004FEAD42E24F40064B1FA81F2202AA4F136
:1036E000020404BFB0FA80F3D218A2F10B02B2F1C7
:1036F0002003A4EB02040CD2C2F1200301FA02F170
:1037000020FA03F341EA030100FA02F0C2F12003B8
:1037100003E000FA03F14FF0000001EBCE71002C42
:1037200001EB0451BDE81040A8BF704701F1C04152
:103730004FF0000001F00041704701EB045110BD53
:10374000491001EB0451BDE810404FEA300002E09F
:103750004FF0000170474FF0120C4A0008BF0042C2
:10376000F6D0B2F5001F28BF704701F000414FF0BE
:10377000000070479CEA445F07D0BDE8104011EAA2
:103780005C0F04BF002100207047012841EB0104B9
:10379000012A43EB030E644598BFE645DFF848C0B5
:1037A000BDE8104031F61CACAFF30080012841EBBE
:1037B0000100012A43EB0302904209D010F5001FDB
:1037C00004BF0020704783F000414FF000007047B5
:1037D00091EA030F4FF0000048BF704703494FF0D4
:1037E000000070470000E0FF120000040000F87FB6
:1037F000094248BF4CF4803C4FF4C0634FEA115279
:1038000003F1010321EA025122F400629A1A48BF2F
:103810006FF0FE0241F48011352A3CD830D0152AD1
:103820001ED3203A0CD90028C2F1200321FA02F05D
:1038300001FA03F218BF42F001024FF0000130E03C
:10384000C2F1000302F1200201FA03F120FA02F2B0
:1038500041EA020100FA03F208464FF0000120E0BD
:10386000C2F1200310B400FA03F401FA03F320FAC2
:1038700002F021FA02F1224610BC43EA000010E0F7
:1038800050EA01324FF000004FF000014FF00042CB
:1038900018BF521C05E04FF001024FF000014FF03D
:1038A00000001CF4803F2CF4803C18BF41F0004124
:1038B000124208BF7047520003D303D0401C41F1AD
:1038C000000170475FEAAC72F8D4FAD1401C41F1B4
:1038D000000120F00100F4E77047704700F5000C8C
:1038E0001CF0FE4F09D0C1104FEA407001F1605149
:1038F00058BF7047A1F1E04170471CF4000F08D099
:103900000146400008BF70474FF000004FEA300109
:103910007047DFF814C0420272F462ABAFF300806C
:1039200040F4E001104670471800000490EA010FCF
:1039300048BF81F0004100F1F882421A3CBF801A72
:1039400089184FEAD0524FF07F4C1CEA410FA2EB8E
:10395000D15318BF9CEA026F00F040804FF0004C3A
:103960004CEA00204CEA012121FA03FC10EB0C0C7C
:1039700023D202F1FF325FEA1C2040EBC25038BF75
:1039800070471CF07F0F4FEA400C18BFBCF17F4F0F
:1039900038BF7047C3F12003994008BF20F00100F1
:1039A000BCF17F4F38BF7047A0F1C0404FF0FF011E
:1039B00041EAD0514FEAC15070474FEA3C00000A3B
:1039C00040EBC25028BF1CF0FF0F4FEA400CE1D083
:1039D00018BFBCF17F4F38BF7047E5E79CEA026F24
:1039E00005D010EA5C0F08BF00F000407047BCEB48
:1039F000410F4FEA400228BF9445DFF828C0F2F497
:103A0000E9AAAFF30080B2EB410F05D012F1807F3D
:103A100008BF70470846704790EA010F58BF7047CB
:103A200001487047010000040000C07F4FF47F0C84
:103A30001CEAD0121EBF1CEAD11392EA0C0F93EAC3
:103A40000C0F00F0A58090EA010F48BF42F480728D
:103A500040F4000C41F400002CF07F4120F07F4046
:103A600000B58142A2EB03020FF2401CACEB504EBA
:103A7000C0F100009EF800E04FEA4E0E00FB0EFC85
:103A800038BF49004FEA2C1C02F5FA020CFB0EF37A
:103A90004FEACE1E4FEA112C4FEAC1210EEB635EB6
:103AA0000EFB0CFC4FEA1C5300FB03114FEA112CD8
:103AB0004FEA01310EFB0CFC02F4807E42EB224205
:103AC0004FEADC4C00FB0C11C14228BF09184CEB3B
:103AD0000333012924BF4EF0020E4EF0804E10EB4E
:103AE000410F24BF4EF0010E4EF0804E08BF4EF045
:103AF000040E4EF008015DF804EB43EBC25018BF12
:103B0000B2F57C0F38BF704741EAC07108BF20F0A2
:103B10000100B2F57C0F38BF704729D512F0F00FC5
:103B20001CBF00F1C04000F000407047008182835C
:103B30008485868788898B8C8D8E8F9192939596BC
:103B400097999A9C9D9FA0A2A3A5A7A8AAACAEB046
:103B5000B2B3B5B7B9BCBEC0C2C5C7C9CCCED1D44B
:103B6000D7D9DCDFE2E6E9ECF0F3F7FAFE0000007B
:103B70004FEA400C0CF1807CBCF17E4F28BF7047AF
:103B8000B0F1C0404FF07F404CBF4010400870473C
:103B900090EA010F0CEAD11348BF42F480726245EB
:103BA00038BF634507D213F47F0F23D080EA0100AA
:103BB00000F0004070474FF0807C1CEB400F98BF36
:103BC0001CEB410FDFF840C032F604AAAFF30080CF
:103BD0004FF0807C1CEB400F02BF1CEB410F0B48E9
:103BE00070471CEB410F0CBF002020F0004040EA62
:103BF000C250704712F47F0F04BF0448704742F070
:103C0000FF004FEAC0507047040000040000C07F6E
:103C100050EA010C00F113801CF5000F58BFBCF5F1
:103C2000000F01D48842704707D710F5000F58BF26
:103C300011F5000F15D488427047894270471CF572
:103C4000000F04D5BCF5000FF7D5814270474FF047
:103C5000807C1CEB400F38BF1CEB410F01D281422E
:103C60007047DFF808C0F1F7A3BE00000900120496
:103C7000C2154FEA002318BF43F0004305D4D2F128
:103C80009E020AD323FA02F070474FEA4001B1F1D5
:103C9000FE4F02D24FF000007047DFF828C04FEA15
:103CA0004001B1F17F4F88BF4CF4803C32F698A9B7
:103CB0001CBF6FEAE0707047AFF300806FEAE070FE
:103CC000704700006800020410F0004218BF404234
:103CD00042F08042B0FA80F18840A2EBC15202F17A
:103CE000786208BF7047410642EB202018BF5FF0A2
:103CF000806C28BF20F001007047000050EA010CE2
:103D000000F113801CF5000F58BFBCF5000F01D463
:103D10008842704707D710F5000F58BF11F5000F04
:103D200015D488427047894270471CF5000F04D5AE
:103D3000BCF5000FF7D5814270474FF0807C1CEB3B
:103D4000400F38BF1CEB410F01D281427047DFF8B2
:103D500008C0F1F72DBE0000090016044FF47F0CD7
:103D60001CEAD0121EBF1CEAD11392EA0C0F93EA90
:103D70000C0F00F04A8090EA010F48BF42F48072B5
:103D80004FF0004C4CEA00204CEA01211A44A0FB01
:103D900001C3A2F50002BCF1000F18BF43F00103FC
:103DA00002F4807CB3F1004F38BF5B0042EB22424B
:103DB000180A40EBC25028BF13F07F0F18BFB2F5AE
:103DC0007C0F38BF704708BF20F00100B2F57C0FB0
:103DD00038BF70470BD582F0FF0212F5803FC8BF95
:103DE000704700F1C040D8BF00F00040704700F5B8
:103DF000000C5FEA4C0C48BF7047B0F1C0404FF078
:103E00007F404CBF40104008704790EA010F0CEA19
:103E1000D11348BF42F48072624538BF634504D273
:103E200080EA010000F0004070474FF0807C1CEBFE
:103E3000400F98BF1CEB410F4FF0030C4CF0806C0F
:103E400032F6C8A8AFF3008012F47F0F1FBF13F43F
:103E50007F0F42F0FF02D005704701487047000015
:103E60000000C07F10B412F47F0F4FEA00204FEA29
:103E7000012110D1B0FA80F400FA04F0A2EB044260
:103E800013F47F0F02F5803218BF41F0004100D0DB
:103E900010BC18BF604740F00040B1FA81F401FA4D
:103EA00004F1A3EB044310BC03F58033604700002A
:103EB00051EA000C00F113801CF5000F58BFBCF54F
:103EC000000F01D48142704707D711F5000F58BF8A
:103ED00010F5000F15D481427047894270471CF5D8
:103EE000000F04D5BCF5000FF7D5884270474FF09E
:103EF000807C1CEB410F38BF1CEB400F01D2884285
:103F0000704781EA000080EA0101DFF80CC081EA15
:103F10000000F1F74DBD00000900160490EA010F02
:103F200048BF81F000413FF508AD421A3EBF82F024
:103F30000042801A89184FEAD0524FF07F4C1CEA99
:103F4000410FA2EBD15318BF9CEA026F4FD04FF044
:103F5000004C4CEA00204CEA012121FA03FCB0EBB2
:103F60000C0C0FD412F0FE0F18BF5FEA4C001DD5E9
:103F7000001240EBC25038BF70471CF03F0F18BF13
:103F800070470BE0A2F101025FEA1C2040EBC25037
:103F900038BF70471CF07F0F18BF7047C3F1200374
:103FA000994014BF401E20F0010070474FEA1223D1
:103FB00016D0004204BF002070474FEA9000B0FACC
:103FC00080FCA2EB0C02CCF1280C60FA0CF093EA16
:103FD000122F04BF00EBC25070474FEAC370704706
:103FE0005FEADC1008BF70474FEAC37070479CEA75
:103FF000026F04D010EA5C0F08BF00207047BCEBD2
:10400000410F4FEA400228BF9445DFF82CC0F1F47D
:10401000E1AFAFF30080B2EB410F06D012F1807F29
:1040200008BF704781F00040704790EA010F48BF19
:104030007047024870470000020000040000C07F83
:1040400000F0004343EAD05323F48073C3F1C1036B
:1040500023F0004117291FD8C3F1200310FA03F100
:10406000C3F1200320F07F4040F4000020FA03F069
:1040700003F0004340EA03000DD00B46590009D37A
:1040800018BF401C06D17FEAE27398BF401C38BFBE
:1040900020F0010070477047182903EB912318BFE7
:1040A0006FF00041013168BF03F0004009D64002C3
:1040B00003F0004000F1010004BF12F0004F20F0B7
:1040C0000100704770470CF00F03092B08BF082050
:1040D00000F05B800A2B0BD0082B18BF704708BF7D
:1040E0001CF0400F0AD04FF000004FF00001704765
:1040F0001CF0400F18BF4FF0004070471CF0100F2D
:1041000008D020F0704300F07F4242EAD3014FEA2A
:104110004370704700F0604021F07F4242EA0002A5
:1041200001F07F4040EA727070474FF0FF0C4CF492
:10413000E06C1CEA11531CBF9CEA030C9445C2BFFF
:10414000DA4201EB02517047002B0DD0BCF1000F99
:104150000FD0002A01F00041A4BF41F0E04141F03E
:104160007F614FF00000704701F000414FF0000008
:10417000704750EA01334FF09B0C18BF4CF0806C35
:1041800070F436AFAFF3008070471CF4801F11D07D
:104190001CF4E02F03D06FEACC31490070474FF098
:1041A0004050EFF3008222F0704242EA000282F3B4
:1041B000008870474FF000007047C800F65E10009E
:1041C0001000000025001E000000FFFF000000009E
:1041D00000000000A500A500A500A500A50011088D
:1041E0000F000A00000000000000000000000000B6
:1041F0000000000000003D001C0000000000140052
:10420000FF00D703000000000000FFFFFFFFFFFFDB
:10421000FFFFFFFFFFFFFFFFFFFF0000FFFF0000AA
:10422000000000000000000000000000000000008E
:104230000000000000003B1800000000000000002B
:10424000000000000000F401000000000000000079
:10425000000000000000000000000000000000005E
:10426000000000000000000000000000000000004E
:10427000000000000000000000000000000000003E
:1042800000006400F65E1000000000000000000066
:10429000000000000000000000000000000000001E
:1042A0000000DC0DB63D0000000000000000000032
:1042B00000000200030000000000000000000000F9
:1042C00000000000000000000000000000000000EE
:1042D00000000000000000000000000000000000DE
:1042E00000000000000000000000000000000000CE
:1042F00000000000000000000000000000000000BE
:1043000000000000000000000000000000000000AD
:10431000000000000000000000000000000000009D
:10432000000000000000000000000000000000008D
:10433000000000000000000000000000000000007D
:10434000000000000000000000000000000000006D
:10435000000000000000000000000000000000005D
:10436000000000000000000000000000000000004D
:10437000000000000000000000000000000000003D
:10438000000000000000000000000000000000002D
:10439000000000000000000000000000000000001D
:1043A000000000000000000000000000000000000D
:1043B00000000000000000000000303132333435CE
:1043C000363738394142434445460000000000007A
:1043D00000000000000000000000000000000000DD
:1043E00000000000000000000000000000000000CD
:1043F00000000000000000000000000000000001BC
:104400000203040506070809000000000000000A76
:104410000B0C0D0E0F00000000000000C1814001D8
:10442000C0804101C0804100C1814001C080410085
:10443000C1814000C1814001C0804101C080410074
:10444000C1814000C1814001C0804100C181400163
:10445000C0804101C0804100C1814001C080410055
:10446000C1814000C1814001C0804100C181400143
:10447000C0804101C0804100C1814000C181400134
:10448000C0804101C0804100C1814001C080410025
:10449000C1814000C1814001C0804101C080410014
:1044A000C1814000C1814001C0804100C181400103
:1044B000C0804101C0804100C1814000C1814001F4
:1044C000C0804101C0804100C1814001C0804100E5
:1044D000C1814000C1814001C0804100C1814001D3
:1044E000C0804101C0804100C1814001C0804100C5
:1044F000C1814000C1814001C0804101C0804100B4
:10450000C1814000C1814001C0804100C1814001A2
:10451000C0804101C0804100C1814000C0C101C3D1
:104520000302C2C60607C705C5C404CC0C0DCD0FD7
:10453000CFCE0E0ACACB0BC90908C8D81819D91B87
:10454000DBDA1A1EDEDF1FDD1D1CDC14D4D515D707
:104550001716D6D21213D311D1D010F03031F13357
:10456000F3F23236F6F737F53534F43CFCFD3DFF17
:104570003F3EFEFA3A3BFB39F9F83828E8E929EBE7
:104580002B2AEAEE2E2FEF2DEDEC2CE42425E52747
:10459000E7E62622E2E323E12120E0A06061A163B7
:1045A000A3A26266A6A767A56564A46CACAD6DAF57
:1045B0006F6EAEAA6A6BAB69A9A86878B8B979BB07
:1045C0007B7ABABE7E7FBF7DBDBC7CB47475B57787
:1045D000B7B67672B2B373B17170B0509091519317
:1045E00053529296565797559594549C5C5D9D5F97
:1045F0009F9E5E5A9A9B5B99595898884849894B67
:104600008B8A4A4E8E8F4F8D4D4C8C4484854587C6
:1046100047468682424383418180401F1C1F1E1FE4
:104620001E1F1F1E1F1E1F004C5555555555A53FDB
:104630007751C1166CC156BF9015CB19A001FA3E37
:10464000AD529C804F7E92BEC4B1B4BD9EEE213E61
:10465000D43888BEE9FAA8BD5CE6C0662339A03C20
:10466000A85B6F48B1C254396BC7F7CA684025B61A
:10467000C59ABD840792E332E44BFD1E2F70A62F2E
:10468000975EC67A0B1D49AC2EC93BAA1ABD0329F9
:104690005022A2C996F5DEA5D5FD559580B7A22278
:1046A0001E616A04878C639FB6A36F91DDC8FE1BF1
:1046B0002B350EDC52C2D618894D4CB5F87789954A
:1046C0006BAC554CB6AFCA91167F3C590B69F78E4F
:1046D000C7C6E941A371E50BADAA5188D9BDA3882E
:1046E0007DDEF39433D5620500004054FB21F93F91
:1046F0003163621A61B4D03D0000601A61B4D03DEC
:104700007370032E8A19A33B0000002E8A19A33B65
:10471000C14920259A837B39A6F810111111813FD8
:10472000D561C119A0012ABF7DFEB157E31DC73E67
:10473000EB9C2B8AE6E55ABE7CD5CF5A3AD9E53DAB
:104740007AFE10111111C13F37D60684F464963FEA
:10475000280356C9226D6D3F0165F2F2D844433FEC
:10476000A69237A0887E143F735360DBCB75F3BEEF
:10477000FE41B31BBAA1AB3F93846EE9E326823FAF
:104780001583E0FEC8DB573F68108D1AF726303FCF
:10479000E9A7F0320FB8123FD47ABF74702AFB3EFB
:1047A000C047010800000020240100005C0100084F
:1047B000E448010824010020C4D400007801000866
:1047C00002040608000000000102030401020304C1
:1047D0000607080900A24A040000000000000000CB
:1047E00001020304060708090000000000000000A1
:1047F000FF000000000000000000000000000000BA
:1048000000000000000000000000000000000000A8
:104810000000000000000000000000000000000098
:104820000000000000000000000000000000000088
:104830000000000000000000000000000000000078
:104840000000000000000000000000000000000068
:104850000000000000000000000000000000000058
:104860000000000001001000000100100000000026
:104870000000000000000000000000000000000038
:104880000100030007000F001F003F007F00FF0032
:10489000FF01FF03FF07FF0FFF1FFF3FFF7FFFFF2A
:1048A0000000000000000000000000000000000008
:1048B0000A000000010000000100000000000000EC
:1048C00000000000000000000000000000000000E8
:1048D00000000000000000010404000205000306BF
:0448E00001040600C9
:0400000508000121CD
:00000001FF
